:100000004DC4000083C4000081C400007FC4000010
:100010007DC400007BC4000079C4000077C40000E8
:1000200075C4000073C400000C94D62D0C94BE2E31
:100030000C941E1A6BC4000069C4000067C4000061
:1000400065C4000063C4000061C400005FC4000018
:100050005DC400000C94B22D59C4000057C40000C8
:1000600055C4000053C4000051C400004FC4000038
:100070004DC400004BC4000049C4000047C4000048
:1000800045C4000043C4000041C400003FC4000058
:100090000C94C2303BC4000039C4000037C40000D7
:1000A00035C4000033C4000031C400000501090656
:1000B000A1018506050719E029E715002501950826
:1000C000750181020507190029EF1500250195F03A
:1000D000750181020508190129059505750191022F
:1000E000950175039101C00660FF0961A1010962D4
:1000F000150026FF0095207508810209631500266A
:10010000FF00952075089102C005010906A10105AF
:100110000719E029E7150025019508750181029569
:1001200001750881010507190029FF150026FF0048
:100130009506750881000508190129051500250196
:10014000950575019102950175039101C0000000AC
:10015000000000000000000000000000000000009F
:10016000000000000000000000000000000000008F
:10017000007E0F00D4FFFFFFC700000078000000E2
:1001800000000000002A2B280000000000000000F2
:10019000000000000000000029000000002C1E34B8
:1001A00020212224342627252E362D3738271E1FBE
:1001B000202122232425263333362E37381F0405E9
:1001C000060708090A0B0C0D0E0F10111213141557
:1001D000161718191A1B1C1D2F3130232D35040535
:1001E000060708090A0B0C0D0E0F10111213141537
:1001F000161718191A1B1C1D2F3130354C09025BBC
:1002000000030100A0FA0904000001030101000934
:1002100021110100012244000705810308000109A2
:100220000401000203000000092111010001222243
:1002300000070582032000010705030320000109D0
:100240000402000103000000092111010001223B0A
:1002500000070584032000011201000200000008CD
:1002600044564D530100010203011C03760069004E
:1002700061006C003A006600360034006300320012
:1002800062003300630000001003530050005F0061
:100290004D0069006E0069000000240356006900EB
:1002A0006B0074007500730020004400650073004B
:1002B000690067006E0020004C004C004300000005
:1002C0000403090401000100010001000100010014
:1002D000010000002152290014001A000800150036
:1002E0001700000022522B0004001600070009002E
:1002F0000A0000000100E1001D001B0006001900BB
:10030000050000000100E000E200E30021522C4162
:1003100000000000010001000100010001000100D7
:10032000010001001C0018000C00120013004C001A
:100330002A0001000B000D000E000F003400000029
:100340002800010000001100100036003700E50011
:1003500052000000000000002A42E6002252500035
:1003600051004F000100007C01000100010001006C
:1003700001000000010035001E001F0020002100C8
:100380002200000001002078237825782778A90032
:100390002F00000001002178247826782878AA0010
:1003A0002F02000001000100010001000100010016
:1003B0000000000001000100010001000100010037
:1003C00001000100230024002500260027002D0045
:1003D0002E00010030002100220023003300000025
:1003E00001000100000030021E001F00200001007B
:1003F00052000000000000004C00270001005000E7
:1004000051004F0001000100010001000100010046
:1004100001000000010035021E021F02200221021D
:1004200022020000010001000100010049004B0010
:100430004A00000001000100010001004C004E00D4
:100440004D000000010001000100010001004C000E
:100450000000000001000100010001000100010096
:1004600001000100230224022502260227022D0298
:100470002E02010001000100010001003302000012
:100480000100010000000100010001000100010065
:1004900052000000000000000100010001005000B7
:1004A00051004F00AA00A900AA00A900AA00A900B3
:1004B000AA00A900AA00A900AA00A9002225282AAA
:1004C0002D3033363A3D4043474A4E5155595C60D2
:1004D00064686B6F73777B7F83878A8E92969A9E10
:1004E000A1A5A8ACAFB3B6B9BCBFC2C5C7CACCCE74
:1004F000D1D2D4D6D7D9DADBDBDCDCDDDDDCDCDC69
:10050000DBDAD9D8D7D5D3D2D0CDCBC9C6C3C1BEFB
:10051000BBB8B4B1AEAAA7A39F9C9894908C8985D0
:10052000817D7975716D6966625E5A5753504C4989
:1005300045423E3B3835322F2C292623FFAA7F55D2
:100540004000010101010101010101020202020258
:10055000020202020303030303030303040404046B
:100560000404040505050505060606060607070733
:10057000070708080808090909090A0A0A0B0B0BEA
:100580000C0C0C0D0D0D0E0E0E0F0F0F1010111187
:10059000111212131314141515161617171818190B
:1005A000191A1A1B1B1C1D1D1E1E1F202021222272
:1005B000232424252626272829292A2B2C2D2D2EB5
:1005C0002F30313232333435363738393A3B3C3DCF
:1005D0003E3F404142434445464748494A4C4D4EC0
:1005E0004F50515354555658595A5B5D5E5F616286
:1005F00064656668696B6C6D6F7072737577787A15
:100600007B7D7E8082838587888A8C8E8F9193956F
:1006100096989A9C9EA0A2A3A5A7A9ABADAFB1B393
:10062000B5B7BABCBEC0C2C4C6C9CBCDCFD1D4D673
:10063000D8DBDDDFE2E4E7E9EBEEF0F3F5F8FAFD15
:10064000FF1E0F0500047F3F1F64321464321478CC
:100650003C1E1E140A05FD377A585A000004E6D6DF
:10066000B4460200210116000000742FE5A3E00645
:10067000AA01E65D003D8889C65436C3174FE4E6FB
:1006800021E04F213B49E126C7E663B1176A98464E
:10069000C3AF9E71F619F315EC0B5CF0B0B910FE08
:1006A00097FD38E2BD40991E527A9E35EE78F9E901
:1006B0009DC06E055C54B2971B8A4989D26151CBAB
:1006C00096677368F63B8BD545236F383A204C47C5
:1006D0005BF7A952735DD0338433BB1F6154DE7F57
:1006E0004B106C57151743DDD779EE01615376CF68
:1006F0000B4DB5C2F380EDEEC46B14D2F6073D3856
:10070000F2E010A921EE80B68BB8FE88BCE531BEC0
:1007100021AD0F2E1D5B5953A8DC72F1B00B15D71C
:1007200082E9665C721DA8A64BD69E5AFA2E35FF4A
:10073000D9D2B300BCA97094C12214E1C16BCAB56F
:100740006C40D26C3DEE2BCB24AFABF77482ED0E38
:1007500082ADC83109AA56A309939CC8774064A406
:10076000F9472E51A5A3DE8EE6ED02E501BC14D8B3
:1007700030B69E6703D33C20FEC7F00DDF5AEAA6D1
:10078000CDE1000D9A60386FB39EC44B677FCBB943
:100790003EC2D957B4FD6E09BB6EB524574F7F21B9
:1007A000821218D3D35DE30A38749DD02BC986EF2B
:1007B0000AF530B47578477C1833588A796E4ABC8C
:1007C000E4849B0DAB9648AB6B101346ECD617FC3C
:1007D000C524D2C339AC910329108CADF6BD17588E
:1007E00063CF95196395F1A02D04BB1431B3CE7777
:1007F000EBA1B296BE442403877F773F8DDDA20E26
:10080000BFDC81A3457E2E4DB831574F8B942EDD32
:1008100096F4C471463F3B354725EDF6A997A19C58
:100820005D423D58B61C01E43AE54FD45CA2375115
:10083000563FF2061E19BF1813C7FABE4C0EEDEC58
:100840001F2820FEED3E78A9FFF93716469EB23DDF
:10085000A672040D2D8AB720241429000000E6F2A8
:100860002B330621FCBB00018204AB0D000099CAAA
:100870001FF7B1C467FB020000000004595A504F33
:1008800052514A4D4B4E2A4C2F300D0E0B0F1A056C
:1008900008050905071811130408120C11241FBEBE
:1008A000CFEFDAE0DEBFCDBF04B603FE18C0809103
:1008B000860490918704A0918804B09189048730C0
:1008C000904BA740B04B59F41092860410928704C5
:1008D0001092880410928904E0E0F8E3099524E07E
:1008E000AAEDB1E001C01D92A638B207E1F711E010
:1008F000A0E0B1E0E0E9F7E602C005900D92AA3D64
:10090000B107D9F70E940A260C94903379CB9C0149
:10091000FB019A9581159F4120F5832F8170B32F9C
:10092000B270AA27732F74706627532F587044270C
:1009300034FF0DC08295807FAB2B09F08062672B5E
:1009400009F08064452B09F0806809950895AB2B68
:1009500009F08260672B09F08460452BB1F3886051
:10096000F4CF80E0F2CF0C94EC310895982F92955B
:100970009F7024E0911102C020E0982F892F869566
:100980008695811511F02E5F982F892F8695820FFD
:100990000895CF93C82FEADF823039F0833049F0D1
:1009A000813069F48D9A8E9802C08E9A8D988F98B6
:1009B00003C08F9A8D988E988C2FCF9108958D9823
:1009C000F2CF80930E040895E4DF80930F0408951E
:1009D00021E030E001C0220F8A95EAF780910F04F0
:1009E000822BF2CF21E030E0A90102C0440F551F55
:1009F0008A95E2F7CA01809590910F048923E4CF8C
:100A00009B01677091E001C0990F6A95EAF763E076
:100A1000369527956A95E1F7B901660F771F260F7E
:100A2000371FFA01E20FF31F40E050E0682F70E03B
:100A30008191DF019B01042E02C0369527950A940F
:100A4000E2F7217021952827292328272E934F5F2D
:100A50005F4F4330510561F708959C01A82FA7709F
:100A600083E0369527958A95E1F7C901880F991F8C
:100A7000820F931FFB01E80FF91F40E050E080E078
:100A8000219130E00A2E02C0369527950A94E2F7AC
:100A900021703327042E01C0220F0A94EAF7822B1B
:100AA0004F5F5F4F4330510559F70895282F862F28
:100AB000903F69F09A3060F4283048F438E0939F12
:100AC000B0011124620F711D4BE753E099CF0895D7
:100AD0009C5F9230E0F7622F70E048E753E0F6CF7A
:100AE000282F903FA1F09A3058F4883080F438E0F5
:100AF000939FC00111246BE773E0820F911DADCF6E
:100B00009C5F923020F468E773E090E0F8CF80E0DB
:100B1000089590910F0421E030E0F90101C0EE0F3B
:100B20008A95EAF7D90102C0AA0FBB1F6A95E2F7BE
:100B3000EA2B01C0220F4A95EAF7892F8E23E8138A
:100B400003C0892F822B40CF2095822F8923FBCF92
:100B50008091120490911104981301C008958F5F41
:100B60008770FACF982F909580910D0489238093F8
:100B70000D040895803E9105D9F1C8F481339105A3
:100B800009F482C048F48932910509F472C08A32AE
:100B9000910509F480C0089589339105E9F0823800
:100BA0009105D1F08533910509F45EC00895843E26
:100BB0009105D9F148F4823E910539F1833E9105C2
:100BC00049F181EE90E00895863E9105C9F1873E96
:100BD000910509F43EC008952091990323702111D5
:100BE00064C020919A0323FF14C089E290E0089525
:100BF0002091990320FD45C030919A0330FF09C030
:100C000024FD24C083EE90E008952091990322FDF5
:100C1000F7CF08952091990322FD44C030919A03A3
:100C200030FD43C024FFF5CF11C020919A0321FF6E
:100C3000F0CF8091990384FD09C087EE90E008957C
:100C40002091990323FFE5CF24FFF7CF80E090E0C8
:100C500008952091990323FD2BC030919A0331FF11
:100C6000E1CF84EE90E008952091990325FFD1CF44
:100C7000BCCF2091990325FD1EC020919A0323FF2C
:100C8000C8CF89E390E008952091990326FFC1CF52
:100C90008AE290E008952091990326FFBACF81E37C
:100CA00090E0089582EE90E0089580EE90E008953F
:100CB00086EE90E0089585E390E008959091990381
:100CC00092FF10C041E0282F2471243009F040E049
:100CD00031E0282F2871283009F030E0431711F057
:100CE0002CE0822793FF10C041E0282F247124318B
:100CF00009F040E031E0282F2871283109F030E078
:100D0000431711F02CE0822730919A0330FF10C076
:100D100051E0282F2171213009F050E041E0282FC7
:100D20002871283009F040E0541711F029E082279B
:100D300031FF10C041E0282F2171213109F040E03E
:100D400031E0282F2871283109F030E0431711F0E5
:100D500029E0822794FD877E08951F93CF93DF9328
:100D600009DFEC01811522E5920708F044C08115E6
:100D700040E5940708F0B5C0883E9105E0F4803E58
:100D8000910560F4853A910570F4049738F481E098
:100D9000219709F080E0C82F50E0D52FCE01DF91D8
:100DA000CF911F9108958D5C9109D0654397B0F361
:100DB000C0E0D0E0F3CFC11580E4D80798F4C115A6
:100DC00090E2D90708F0A3C0CE019A9581159F4102
:100DD00078F78D2F73DF182FCE019927CBDEEC012A
:100DE000D12BDCCFCE019927C5DECC27DF70C82BF5
:100DF000D92BD06AD3CF803842E59407C8F5803626
:100E000052E5950708F058C0C03482E5D807D0F401
:100E1000C03292E5D90708F048C08C2F8695869598
:100E200020E2829FC0011124C37021E030E0A901BB
:100E300002C0440F551FCA95E2F7EA01C82BD92B0F
:100E4000DD68ACCF8C2F86958695877050E2859FA4
:100E5000C0011124C37021E030E0A90102C0440F99
:100E6000551FCA95E2F7EA01C82BD92BDC6896CF4B
:100E7000803C52E5950768F4C03A82E5D80708F44B
:100E800097CF8C2F8F711ADFC82FD0E0DC2FCC27A3
:100E900085CF805C9245809708F08ACFDC2FCC27E5
:100EA000CC27DF71C06FD06A79CFCF71D0E0DC2F53
:100EB000CC27C16FD06A72CF86958695877020E265
:100EC000829FC0011124C37021E030E0A90102C05B
:100ED000440F551FCA95E2F7EA01C82BD92BDA68EF
:100EE0005DCF8F71EBDE93E0CC0FDD1F9A95E1F7BC
:100EF000CC27DF70282F30E084FF05C050E1859FAC
:100F0000900111243327C22BD32BD06947CF8D2FCB
:100F10008F71D4DE182FCE0199272CDEEC01D12B56
:100F2000D0623CCF80E00895F894E82FE295EF700E
:100F3000F0E041A18F7021E030E0B90102C0660FFE
:100F4000771F8A95E2F7CB01962F9095942391A372
:100F500092A1892B82A37894089581E08093330332
:100F600008950895CF92DF92EF92FF921F93CF934F
:100F7000DF93172FE82FF0E0EF5BFA4F71110CC0F1
:100F8000E4918E2F7E2F6E2FDF91CF911F91FF90D6
:100F9000EF90DF90CF900895E62EF12CC72ED12C44
:100FA000F491EF2F86E0689F90011124CFEFD0E0FD
:100FB000C901BE010E946F31AB01EE0CFF1C65E55B
:100FC000649FC001659F900D1124E81AF90A6E2DE7
:100FD000660F6E0D7E01EC18FD08FE9DD001FF9D91
:100FE000B00D11248B2F169F70011124EF2CFF24BC
:100FF0006E01CE18DF087601FE9D6001FF9DD00CCA
:1010000011247E01E61AF108B701169F7001179F9F
:10101000F00C1124EF2CFF24CE19DF09FC9F700186
:10102000FD9FF00C11247F2D43305105C1F02C3F62
:10103000334058F441305105B1F04230510509F0C8
:10104000A2CFEB2F8F2D7F2F9ECF4430510571F013
:101050004630510509F497CF7B2F8D2D94CF7D2DF0
:10106000EB2F8F2F90CF7F2FED2D8DCFEF2D7B2F5F
:10107000F8CFCF93982F762F842FC22F692F72DF4E
:10108000472F282F80911201C81B8C2F90E009D385
:10109000CF91089580910404843028F48370846093
:1010A0008093040408958C3AE8F38370886AF8CF3B
:1010B000CF938091040480FF03C03DD5CF91089564
:1010C000C091140180911501C817B8F780911201E1
:1010D0009C2F981B892F20E040E060E090E0E1D257
:1010E000CF5FF0CF0F931F93CF93DF93D82F162F9F
:1010F000042F80910404C091140180FD10C0DF9181
:10110000CF911F910F910895809112019C2F981BF0
:10111000892F202F412F6D2F90E0C3D2CF5F809178
:101120001501C81788F3C4DFEACFCF93DF93EC0132
:10113000209107049C81892F817090FD822F692F57
:10114000627091FD622F492F447092FD422FCADFD9
:101150008C8190E00196877099278C83DF91CF91E5
:101160000895982F762F842F2091040420FF07C024
:10117000692FF8DE962F672F482F892FB3CF089558
:10118000CF93DF93EC01E4E0F4E0438162818C8152
:10119000E8DF8C818F5F8C83DF91CF910895E1E050
:1011A000F4E011828281846082830895E4E0F4E0B7
:1011B00080818E7F8083F3DFE1E0F4E082818160D3
:1011C000828376CFCF93DF93EC01EC81F0E0F5954D
:1011D000E795E454FB4F4491E4E0F4E062818181BF
:1011E000C0DF8C818F5F8C83DF91CF910895EF9268
:1011F000FF921F93CF93DF93EC0110E0EE24EA946B
:10120000F12C60911601161768F052DF8C819A81DB
:1012100090FF1DC08F5F8C83DF91CF911F91FF9056
:10122000EF90089520911401210F3327331F70E0B0
:10123000C7010E94D331962F8C81409107046091A1
:101240000604199F800D112414DF1F5FDACF81502F
:10125000E2CFA0E0B0E0EFE2F9E00C948C31EC01D9
:101260008A8101E080FD0FEF8C81811109C001307E
:1012700019F48091160181508093E70281E08C83FC
:1012800010E0809116011817B0F012DF9091E7027C
:10129000013009F051C0809116018150911519F06B
:1012A0008FEF890F91E08093E7029C83CDB7DEB783
:1012B000E9E00C94A8318091140190911201891BEE
:1012C000810F20E040E060E090E0EBD194E0E92E77
:1012D000F12CB12CC12ED12C8091E7028B0D8931DC
:1012E0002CF168E10E94C631892F082E001C0008ED
:1012F0008C150D04A1F4809114019601280F311D65
:10130000409107046E2D6403A00111245595479563
:10131000559547956091060480910504AADEB00EAC
:1013200081E0E81AF108C1F61F5FABCF87FFDDCF80
:1013300090911601890FD9CF892F90E00196609185
:10134000160170E00E94D331982FADCF1F93CF9339
:10135000DF93EC018C81811109C081E08C831092B4
:10136000E60292E09093060180930501109114012A
:1013700080911501181740F110E0609116011617C1
:1013800078F196DE809105019091E602980F909396
:10139000E60220910601280F20930601121654F44C
:1013A000209116012150330B092E001C00089217C2
:1013B000030634F0819580930501813009F41C8285
:1013C000DF91CF911F91089580911201912F981B69
:1013D000892F20E040E060E090E063D11F5FC8CF3C
:1013E000E12FF0E070E0CF010E94D3312091140191
:1013F000820F9091E602092E001C0008E917F00503
:101400009CF090910601092E001C00089E170F0603
:101410005CF0282F30E04091070460910604809131
:10142000050427DE1F5FA9CF90911201891B20E0E0
:1014300040E060E090E035D1F5CFA6E0B0E0E3E237
:10144000FAE00C948D318D839E83AD81BE8114961C
:10145000FC912F2F30E0D9010E9481339B01AC0118
:101460000E944F336B017C0180E290E09C012F1BB6
:101470003109F901A5E5B0E0A70196010E944F33BB
:1014800069837A838B839C839F01DF010E940332EF
:101490009B010E9409329B01AC012C0D3D1D4E1D8C
:1014A0005F1D69817A818B819C810E945F33022F4D
:1014B00030E00A3240F5A901440F551F420F531F77
:1014C00055954795142F1095F12C85E5E82EE01AD7
:1014D00080911601F81628F1EBDDAD81BE811496DE
:1014E0009C9181E0911519F0903219F48FEF80935F
:1014F000040180910401890FED81FE818483269689
:10150000E8E00C94A93185E590E0821B930BAC01D7
:10151000440F551F480F591F57FFD2CF4F5F5F4FE2
:10152000CFCF8E2DF1FC802F209114012F0D33276A
:10153000331F412F609106049CDDF394C9CF0F93B4
:101540001F93CF93DF93EC0100E010E09091160120
:101550000917110564F0ACDD8C8190E00196817073
:1015600099278C83DF91CF911F910F9108954C8122
:10157000809114019801280F311D6091060480911B
:10158000050496950917110544F4411541F0409161
:1015900007046FDD0F5F1F4FD9CF4115C1F340E046
:1015A000F8CFFB01811520E2920728F4811541E074
:1015B000940738F408959C0130522115304348F0C7
:1015C0000895392F94FF02C03295307F2081232B5C
:1015D000208399270895462B22FF0FC0982F9295BC
:1015E0009F708F70892B962F92959F706F70692BCB
:1015F000942F92959F704F70492B982F9623961396
:1016000009C050E04095509590E04823592381E06F
:10161000452B09F080E0089590910D03292F30E0CB
:1016200070910E03A9014F5F5F4F437055277417E8
:10163000150689F0255F3C4F60FB87F9F90184832B
:101640009F5F937090930D0380910B038F5F809346
:101650000B0381E0089580E0089521EF611101C03E
:1016600024EF30B32F7081E090E001C0880F2A95FD
:10167000EAF7982F9095932390BB91B3892B81BB68
:10168000089521EF611101C024EF8FB190E02F7018
:1016900002C0959587952A95E2F7817008956E9A14
:1016A0000895FC01EE0FFF1FE80FF91FEA5DFD4FE3
:1016B0006183408322830895FC01680F791F8FEFB7
:1016C00041E39191892728E030E0982F990F87FF17
:1016D00009C0892F842721503040B9F7E617F70752
:1016E00081F70895892FF7CF0F931F93CF9301E0D0
:1016F00010E0082E01C0000F0A94EAF7C0910C0414
:101700009C2F9023911108C063D9C027C0930C046B
:10171000CF911F910F91089565D9F7CF9091F00364
:1017200089029001112437FF03C08093F0030895CC
:101730002F3731051CF4980F9093F00308959C0106
:1017400080E090E0F901E80FF91FE491E41307C08D
:1017500091E08927F901E80FF11D84910895019620
:10176000861780F380E0089580914603811569F023
:10177000E0916E03F0916F03309739F00190F081A2
:10178000E02D309711F00995089580E0089590912B
:101790007301913021F49091990397FD0CC0EEED07
:1017A000F1E09191891302C0DF011E9251E0E43E05
:1017B000F507B9F70895E82FE695E695E695803F99
:1017C000C8F7F0E0EC51FE4F877021E030E0A9014E
:1017D00002C0440F551F8A95E2F7CA018095928195
:1017E0008923828308958091720108952FB7F89418
:1017F000609122027091230280912402909125022F
:101800002FBF08950F931F9380914603811521F0F8
:10181000EDDF1F910F910895E9DF009142031091D0
:1018200043032091440330914503600F711F821FD1
:10183000931FEFCF08950895FC019B01809118023A
:10184000909119028617970740F0672B29F4809131
:10185000E8008E778093E800C90140E0009741F4EA
:10186000411106C08091E80082FF2FC080E00895FA
:1018700020912A032115A9F12530A9F12091E80032
:1018800023FD2DC02091E80022FDECCF2091E8003F
:1018900020FFE4CF3091F3002091F200009719F07F
:1018A0002830310558F041E02830310509F040E09A
:1018B0002091E8002E772093E800D0CF419140930B
:1018C000F10001972F5F3F4FE9CF80912A038115E7
:1018D00041F0853041F08091E80083FFC3CF81E083
:1018E000089582E0089583E008958091120287FFB1
:1018F00013C08091E80082FF06C08091E8008B77DA
:101900008093E800089580912A038111F2CF089511
:1019100080912A038115D9F38091E80080FFF8CFE8
:101920008091E8008E77ECCF2091E4003091E500C3
:1019300095E6A9012091EC00822F817020FF06C05E
:101940008091E80080FF06C080E008952091E800C3
:1019500022FD1AC080912A03811589F0853089F013
:101960008091EB0085FD0FC02091E4003091E500EF
:1019700042175307F9F29A95E1F684E0089582E060
:10198000089583E0089581E00895E8EDF0E0808116
:101990008E7F80831092E2001092DA001092E100B4
:1019A000A0EEB0E08C9181608C9380818F778083F2
:1019B00019BCA7EDB0E08C918E7F8C9380818F7ED7
:1019C0008083109211020895E0916E03F0916F03ED
:1019D000309739F00284F385E02D309711F060E202
:1019E00009950895982F9093E900891771F07091E7
:1019F000EC002091ED005091F00021FD09C09F5FA7
:101A0000973089F78093E9000895762F242F50E0CE
:101A10003091EB003E7F3093EB003091ED003D7F45
:101A20003093ED003091EB0031603093EB00709318
:101A3000EC002093ED005093F0002091EE0027FD84
:101A4000DECF0895A0E0B0E0E8E2FDE00C948D3137
:101A5000C8EDD0E088818F7E8883E7EDF0E080815B
:101A60008160808384E082BF81E08093110288815D
:101A70008E7F888302EE10E0F80110821092DA0067
:101A800081EEC82ED12CF601108288818F77888351
:101A900088818068888388818F7D888319BC1092B3
:101AA0002A03109210021092F60210920F0290EE8A
:101AB000E92EF12CF70180818B7F80838881816002
:101AC000888342E060E080E08DDFF60180818E7FD8
:101AD0008083F80180818160808380818860808339
:101AE000F70180818E7F8083888180618883CDB774
:101AF000DEB7E8E00C94A931E09112049091110452
:101B000029E0E91302C080E00895AE2FB0E02E9FD7
:101B1000F0011124ED5EFB4F3181361306C0308198
:101B2000381303C03581341304C0FD013196E770CA
:101B3000E8CF81E008953EB13F7B2EB120644FB7DE
:101B4000F89486E292E0FC010196508168E02EB99B
:101B5000000000C057FF3EB9550F000000C000C094
:101B600000C03EB900C06A9591F752E08E369507E5
:101B700051F74FBF8FE594E00197F1F700C00000E7
:101B8000089581E08093E00080E28093D800109275
:101B9000C9008FE19EE40197F1F700C0000087E0E3
:101BA00090EBDC018093860490938704A0938804D3
:101BB000B093890488E19CE00FB6F894A8958093CF
:101BC00060000FBE90936000FFCF0F931F93CF93E1
:101BD000DF938B01EA0190912A03943051F58093B1
:101BE000E9008FEF9091E80095FD06C095ED9A957C
:101BF000F1F700008A95B1F78091E80085FF19C0E0
:101C000093DE811111C08091E80085FD06C08091AE
:101C1000E8008E778093E800F3CFF80181918F017F
:101C20008093F100219779F78091E8008E77809377
:101C3000E800DF91CF911F910F910895792F6032C5
:101C400029F440E250E0682F82E0BFCF0895CF939F
:101C5000DF93D82FC92F48E050E0682F792F81E01B
:101C6000B4DF88E0ED2FFC2FAAE1B2E001900D92E5
:101C70008A95E1F7DF91CF910895BC0140E250E0F1
:101C800084E0A3CFA0E0B0E0E8E4FEE00C948B3168
:101C9000F82EE92EB62EA72E8A0180910E029AE028
:101CA000C92ED12C8A3018F0CC24C394D12CC1E099
:101CB000D0E06B2D7A2D8F2D9E2DF8010995811185
:101CC00016C02196CC16DD0694F0CC9FC001CD9FA6
:101CD000900D900D112420E030E045E34A95F1F796
:101CE00000002F5F3F4F28173907B9F7E2CFCDB774
:101CF000DEB7EAE00C94A7311F93CF93DF93C62F92
:101D0000122F632F8330D0F4CA30C0F44830B0F4BF
:101D100090E1C99FE0011124C40FD11DC40FD11D52
:101D200090EA899FC00DD11D1124CE0189960E9491
:101D3000FE32612FCE018A960E94FE32DF91CF9152
:101D40001F9108950F931F93CF93DF93962F142F16
:101D5000022F632F833018F5923008F528E0829F18
:101D6000E001112434E0939FC0011124C80FD91F52
:101D7000C75FDD4F81E084279E01280F311D280FAA
:101D8000311DC9010E94FE3281E090E0111102C0B4
:101D900083E090E0602F8C0F9D1F0E94FE32DF9148
:101DA000CF911F910F9108958091100490910D048F
:101DB000892B90917301913059F59091990397FF78
:101DC00027C08093E50140E250E06EE473E084EECA
:101DD00091E00E94B032892BD1F080E2E4EEF1E094
:101DE000AEE4B3E001900D928A95E1F7E0916E03C5
:101DF000F0916F03309759F00480F581E02D309712
:101E000031F086E08093E40184EE91E00995089535
:101E10008093DC0148E050E060E773E08CED91E0F6
:101E20000E94B032892B99F388E0ECEDF1E0A0E755
:101E3000B3E001900D928A95E1F7E0916E03F09185
:101E40006F03309721F30280F381E02D3097F9F290
:101E50008CED91E0DBCF811531F090910D04892B51
:101E600080930D04A1CF0895811531F09091100455
:101E7000892B8093100498CF0895811519F00E9442
:101E8000B20592CF0895811539F080959091100494
:101E900089238093100488CF08958091FD038115D4
:101EA00021F082E2F0DF1092FD030895CF93C82F56
:101EB000811509F463C08CEF8C0F813A08F060C083
:101EC00080917301813031F1EEEDF1E084EE91E02B
:101ED0002191C217C9F18E179F07D1F78091730125
:101EE0008130B1F1AEEDB1E0EFEF80E09D91C91727
:101EF00009F443C0EF3F19F4911101C0E82F8F5F3F
:101F00008630A1F7EF3FC9F10E2E000CFF0BE45213
:101F1000FE4F32C08091990387FFD6CFEC2FE69514
:101F2000E695E695F0E0EC51FE4F828190E04C2F73
:101F3000477021E030E002C0220F331F4A95E2F7DC
:101F400082239323892B21F08C2F21DC2DDFC6CF18
:101F50008091990387FFC6CFEC2FE695E695E6952D
:101F6000F0E0EC51FE4FC77081E090E001C0880FB7
:101F7000CA95EAF7C281C82BC28316DFCF910895B4
:101F800080E28C0F8830D0F7C77081E090E001C00C
:101F9000880FCA95EAF7C0910D04C82BC0930D04B1
:101FA000ECCFCF93DF93EC01805E9109089720F08E
:101FB00064E37FE0209711F46BE27FE0CE010E94A2
:101FC00087048C2F73DFDF91CF910895811531F055
:101FD0009CEF980F913A18F4DADBE6CE089590E280
:101FE000980F9830D8F7877091E001C0990F8A95C3
:101FF000EAF7892F0E94B205F0CFCF93DF93EC016F
:10200000E5DFCE01805E9109089720F063E47FE070
:10201000209711F46DE37FE0CE010E948704DF91E9
:10202000CF9108951F93CF93DF93182FEB013EDFDD
:10203000209731F4812FCADFDF91CF911F9108954E
:102040008FE99FE00197F1F700C000002197F0CFE2
:1020500010920D0480917301813071F48091990385
:1020600087FF0AC0E6EEF1E08EE1DF011D928A955E
:10207000E9F71092100498CEEEEDF1E086E0F5CF8E
:10208000E7DF2FEF84E39CE0215080409040E1F7B0
:1020900000C0000088E19CE00FB6F894A8958093FA
:1020A00060000FBE90936000FFCFAAE2B0E0EBE5C6
:1020B000F0E10C94923182E192E0FC0101962091D2
:1020C000F100208322E08A319207B9F78091130250
:1020D000893009F457C0C8F4823009F4B2C08330A3
:1020E00009F482C0813081F18091E80083FFE6C06D
:1020F00080911202909113029A3008F0DFC0E92F0C
:10210000F0E0EE56FC4C0C94E6318A3009F489C0BC
:102110008B3051F780911202813231F78091160293
:1021200090911702892B01F78091E800877F8093B7
:10213000E800DBDB81E090911402911101C080E0A6
:102140008093730185DFD0CF80911202813A61F6CE
:102150008091E800877F8093E8008091160290913B
:102160001702892B59F060E080E090E070E064DBBA
:102170008091E8008B778093E800B6CF68E08AE131
:1021800092E0F4CF80911202813209F0ADCF8091BC
:102190001602909117028D7F892B09F0A5CF8091AF
:1021A000E800877F8093E8008091E80082FF17C0F5
:1021B0009091F3008091F200029731F48091F10048
:1021C000813011F0863021F48091F100809372010A
:1021D0008091E8008B778093E80087DB85CF809142
:1021E0002A038111E1CF80CF80911202813A09F058
:1021F0007BCF8091160290911702892B09F074CF42
:102200008091E800877F8093E8008091E80080FF5C
:10221000FCCF809173018093F1008091E8008E776C
:10222000DACF80911202813209F05ECF8091E8000E
:10223000877F8093E80059DB8091150280937101BC
:1022400053CF80911202813A09F04ECF8091E8007D
:10225000877F8093E8008091E80080FFFCCF809129
:102260007101D9CF803889F0823841F5809116020A
:102270008F70873018F58093E9008091EB0085FB23
:10228000882780F91092E90006C08091F602880F35
:1022900090910F02892B9091E800977F9093E8002E
:1022A0008093F1001092F1008091E8008E7723C0B6
:1022B000811116C080911402813009F18091E800EB
:1022C00083FF0AC08091E800877F8093E8008091B7
:1022D000EB0080628093EB00AA96E3E00C94AE31B1
:1022E000823061F780911402811581F01092E9002B
:1022F0008091E800877F8093E800F7DADFCF81E004
:10230000933009F080E08093F602F0CF80911602BE
:102310008F702FEF280F263088F68093E9002091E8
:10232000EB0020FFE3CF933031F48091EB0080622B
:102330008093EB00DBCF9091EB0090619093EB00EA
:1023400021E030E0A90102C0440F551F8A95E2F751
:102350004093EA001092EA008091EB008860E8CF99
:102360008111ACCF109114021F778091E300807827
:10237000812B8093E3008091E800877F8093E800C1
:10238000B4DA8091E80080FFFCCF8091E3008068A0
:102390008093E30083E0111101C082E080932A035F
:1023A0008DCF8058823008F089CF809114029091AF
:1023B00015028C3D53E0950791F583E08A838AE20C
:1023C00089834FB7F894DE01139620E03EE051E296
:1023D000E32FF0E050935700849120FF03C08295D3
:1023E0008F703F5F8F708A30C0F0895C90E08D9372
:1023F0009D932F5F243161F74FBF8091E800877F65
:102400008093E8006AE270E0CE01019615DA8091CF
:10241000E8008B778093E80051CF805DE7CF292FCC
:1024200033272330310509F44EC078F521303105CA
:1024300009F488C08BE590E0EDEFF1E02230310542
:1024400009F03CCF2091E800277F2093E8002091FD
:102450001802309119028217930708F49C0140E09A
:102460002115310509F073C0411171C08091E80058
:1024700082FDCDCF80912A03811549F2853039F252
:102480008091E80083FFF2CFC2CF80911602909135
:1024900017022132310509F446C02232310509F014
:1024A0000DCF8330910508F009CFFC01EE0FFF1F1F
:1024B000E057FE4F0190F081E02D83579E4FDC01E5
:1024C0008C9190E010C09C013327823021F12330A1
:1024D000310568F4232BB9F4E0ECF2E0E4918E2F9F
:1024E00090E0E0ECF2E0009709F4E8CEABCF2330C7
:1024F000310509F0E3CEEAE6F2E0E4918E2F90E0B8
:10250000EAE6F2E0F0CFEAE9F2E0E4918E2F90E023
:10251000EAE9F2E0E8CFE8E8F2E0E4918E2F90E01B
:10252000E8E8F2E0E0CF8330910508F0C7CEFC0187
:10253000EE0FFF1FEA56FE4F0190F081E02D89E07B
:1025400090E080CF82E190E0E8E5F2E07BCF8091FF
:102550002A03811509F45BCF853009F458CF8091A7
:10256000E80083FD54CF8091E80082FD7FCF809109
:10257000E80080FF75CF9091F3008091F200211563
:10258000310519F08830910550F041E0089709F0C5
:1025900040E08091E8008E778093E80061CF44911D
:1025A0004093F1003196215031090196E8CF8038EF
:1025B00009F084CE8091E800877F8093E8008091C5
:1025C00010028093F10070CE811178CE1091140228
:1025D000123008F073CE8091E800877F8093E80086
:1025E0001093100282D91115D9F084E080932A0348
:1025F00042E061EC81E0F6D942E261EC84E0F2D99C
:1026000042E261EC82E0EED942E260EC83E0EAD99A
:1026100080912A03843051F482E0809374014ECE7D
:102620008091E30087FDE1CF81E0E0CF81E0F5CF4D
:10263000A0E0B0E0EEE1F3E10C948631D82EFA018F
:10264000522EC32E780198E08902E0011124EF2B6D
:1026500079F5FE01EF5CFE4F86819781892B09F0A9
:102660004DC0E114F10411F1FE01EF5CFE4F8381D6
:10267000A82EB12CE816F10408F45701CF5CDE4F08
:102680006C817D81AB0149595B4F04E610E09501F7
:1026900082E30E94293097FD2BC06C817D816959AE
:1026A0007B4FA501852D9C2D0E94BD3281E021C06C
:1026B000DE01AF5CBE4F8C91A82EB12C481751059E
:1026C00008F45A01FE01EF5CFE4F81809280C40144
:1026D00089599B4F3C01A5010E94BD3204E610E0E0
:1026E0009501A301682D82E30E94DD2F97FFB1CFF2
:1026F00080E0CDB7DEB7EFE00C94A231D092670452
:1027000060913201709133012091310130E0AB01D1
:1027100049595B4F04E610E082E30E94DD2F97FFEA
:10272000A0CFE6CFA1E0B0E0E8E9F3E10C9483317B
:10273000762E4A015901680101E010E09E012F5FE9
:102740003F4F40E050E060E070E072DF182F8115ED
:10275000A9F1F401208031804280538047D86980FC
:10276000621973098409950964367105810591051B
:1027700030F4B701C6010E945C0B8615F9F08701A1
:10278000950140E050E060E070E0872D51DF082FB8
:10279000B701C6010E945C0B10E086110AC0102F21
:1027A000117000FF06C022D8F40160837183828318
:1027B0009383812F2196E2E10C949F31A701B6010A
:1027C000C5010E94BD32F5CFA5E0B0E0EAEEF3E12D
:1027D0000C948D316B0185E0E82EF12C09E614E0B4
:1027E0009E012F5F3F4F4EE353E062E081E09ADFAE
:1027F000811549F095E0FE013196A9E3B3E001901F
:102800000D929A95E1F795E0E9E3F3E0D6010190A6
:102810000D929A95E1F72596E8E00C94A931A8E08D
:10282000B0E0E5E1F4E10C948F3188E0E82EF12C82
:102830000FE614E09E012F5F3F4F45E353E064E055
:1028400083E070DF182F8115C1F190916E048091A3
:102850003403981791F1F12C9091720480917104D6
:10286000891729F1E92FF0E0E559FB4F608567FBF7
:10287000662760F980859F5F9370909372049091B2
:1028800070049F5F909370048F770E940C0BF82E5A
:102890008111E2CF00E010E020E030E040E050E0C5
:1028A00060E070E085E0C4DE1F2D182302C0F11047
:1028B000F1CF80916E0480933403812F2896E6E057
:1028C0000C94AB31A4E0B0E0E8E6F4E10C948D3177
:1028D000C0902F03D0903003E0903103F09032038A
:1028E0000E94F60B6C197D098E099F0911E0643670
:1028F00071058105910518F10E94020CDC01CB01E4
:102900000296A11DB11D89839A83AB83BC8300E02D
:1029100010E020E030E044E050E0BE016F5F7F4F08
:1029200086E086DE182F811551F00E94F60B609329
:102930002F03709330038093310390933203812FE0
:102940002496E8E00C94A9318F929F92AF92BF92A7
:10295000FF920F931F93CF93DF93CDB7DEB72B97E3
:102960000FB6F894DEBF0FBECDBF88E0E4E0F4E020
:102970008E010F5F1F4FD80101900D928A95E1F7EC
:1029800020910104909102048091030429879A8781
:102990008B87F82E80902B0390902C03A0902D0312
:1029A000B0902E030E94F60B681979098A099B09D9
:1029B000F02FE12F643671058105910510F4F114B3
:1029C000B1F000E010E020E030E04BE050E06F2F8D
:1029D0007E2F87E02DDE811569F00E94F60B609353
:1029E0002B0370932C0380932D0390932E0310924E
:1029F000030481E02B960FB6F894DEBF0FBECDBF67
:102A0000DF91CF911F910F91FF90BF90AF909F905A
:102A10008F9008950F931F93CF93DF93833028F502
:102A20006A3018F5483008F520E1629FE001112472
:102A3000C40FD11DC40FD11D30EA839FC00DD11D1D
:102A40001124CE0189960E94DD32082F10E0102F4C
:102A50000027CE018A960E94DD329801282BC901F9
:102A6000DF91CF911F910F91089580E090E0F8CF12
:102A7000FF920F931F93CF93DF93F42E833070F563
:102A8000623060F528E0829FE001112434E0639F0A
:102A9000B0011124C60FD71FC75FDD4F81E0842727
:102AA0009E01280F311D280F311DC9010E94DD3202
:102AB000082F10E0102F002781E090E0F11002C0F5
:102AC00083E090E08C0F9D1F0E94DD329801282B3F
:102AD000C901CDB7DEB7E5E00C94AC3180E090E001
:102AE000F8CF20914A0330914B03232BC9F4703F58
:102AF00039F4603FA9F48091480390914903089507
:102B00007A3038F4683060F4833050F4462F672F01
:102B100081CF7D3F41F4623018F441E0833050F0C2
:102B200080E090E008957C3FD9F76230C8F78330A9
:102B3000B8F740E09DCFA0E0B0E0E1EAF5E10C9409
:102B40008E317C0100910F0480910E04082BC2E0AD
:102B5000D0E010E0C8010C2E02C0959587950A942C
:102B6000E2F780FD09C02197A8F7D12C8D2DCDB7B4
:102B7000DEB7E7E00C94AA31DC2EB7018C2FB1DF71
:102B80000E94AD06019779F3F1CF0F931F93CF9376
:102B9000FC0187819085009789F4858100811181EE
:102BA000811581F0611571F0C801C5DFC82F682F4C
:102BB000C8010E945605B8018C2F93DFCF911F9159
:102BC0000F910895C8010E947005C82FF4CFCF93CC
:102BD000DF93D82FC92FAFDF6D2F7C2F82DF0E94AC
:102BE000AD06DF91CF910895FC0184818115B1F08C
:102BF000878190850097A1F00E94AD06282F9295BD
:102C00009F709630B9F080F4925F9F70923030F4EC
:102C1000203FD1F058F481E0283E58F080E008953C
:102C200080819181D4DFEACF9A5FEFCF81E0243FAA
:102C3000A9F7089591E0813F09F090E081E0283EF6
:102C400008F080E0892B089581E00895382F292F1E
:102C5000CB01A32FB22F8F3A21E09207A105B10536
:102C600020F48F5A9D4F0C94DD3280E0089585E268
:102C700090E00E94DD32833F89F486E290E00E947A
:102C8000DD32893059F487E290E00E94DD3291E034
:102C9000813809F090E0892F8170089580E0FCCFA1
:102CA000A0E0B0E0E6E5F6E10C948C31EC0188811F
:102CB000811509F1813009F045C08981813051F4D5
:102CC0008A81239660E570E0893311F060E070E05E
:102CD000A9D9EDCF823021F48A812396E7D8E7CFB6
:102CE000833021F48A81239671D9E1CF843041F079
:102CF00022968111DCCFCDB7DEB7E9E00C94A83184
:102D00008A81239620E030E09AE0682F6053770BA9
:102D1000AB016A30710560F02115310551F3EFE91F
:102D2000FFE03197F1F700C0000021503109F4CFE6
:102D3000929FB001939F700D11249A01260F371FA7
:102D40008991E3CFE82FF0E0E358FE4FB490282FAD
:102D500026952695269530E0F901E359FE4FE4903B
:102D60008770F12C082E02C0F594E7940A94E2F7DC
:102D7000E0FAEE24FF24E0F8F901E35AFE4FC49094
:102D8000D12C082E02C0D594C7940A94E2F7C0FA59
:102D9000CC24DD24C0F8F901E35BFE4F049110E080
:102DA00002C0159507958A95E2F701701127E11485
:102DB000F10411F081EE7AD8C114D10411F086EE3D
:102DC00075D860E070E08B2D2DD9C114D10411F0BD
:102DD00086EEFCD8E114F10411F081EEF7D801156C
:102DE000110521F060E070E08CE21CD921965FCFE4
:102DF000A6E0B0E0EEEFF6E10C948E3105EA13E0C8
:102E000081E2E82E82E0F82E98E0D92E46E050E0EC
:102E1000B701CE0101960E94CD32F8018D2D11929D
:102E20008A95E9F7B8016C5F7F4F89819A810E948A
:102E3000D10AF80191838083B8016B5F7F4F8B814A
:102E40009C810E94D10AF801938382838D818683BD
:102E50008E818783F6E0EF0EF11C085F1F4F81E53E
:102E6000E81682E0F80691F62696E7E00C94AA317F
:102E7000A6E0B0E0EEE3F7E10C948631A0902803E1
:102E8000B090290381E090E0909329038093280378
:102E900034EAE32E34E0F32EC12CD12C10E03601BD
:102EA00000E015C0F40125913591452D602F812F4B
:102EB0000E947C0E22E0820E911C539438E0531243
:102EC000F1CF88E0680E711C0F5F0A3049F0C30132
:102ED000880F991FDC01AC53BD4F4D01512CE2CF3F
:102EE000F7012591359141E060E0812F0E94A20E0B
:102EF000F70132962591359140E060E0812F0E94E4
:102F0000A20EF70134962591359141E061E0812FC1
:102F10000E94A20EF70136962591359140E061E0BE
:102F2000812F0E94A20EB8E0EB0EF11C1F5F20E57E
:102F3000C20ED11C133009F0B2CFFE01319686E0EB
:102F4000DF011D928A95E9F701E212E07F0146E078
:102F500050E0B801C7010E941C330A5F1F4F0135C2
:102F6000B2E01B07A1F7B0922903A092280326968E
:102F7000EFE00C94A231A0E0B0E0E1ECF7E10C94BA
:102F80008531FC016280448081E08483ECEBF4E0D5
:102F90007490EBEFF4E0E491C0910704C695C1583A
:102FA000D0E0CC0FDD1FCD2FDD27812C35E0932E17
:102FB000AA24AA94B12C55245A94E719EE2EF12C88
:102FC00080911601881638F00E945808CDB7DEB7F8
:102FD000E0E10C94A131C82CD12C83E0681658F4A0
:102FE000989CF0011124E259FD4F809105048083E3
:102FF00080910604818341101CC09C9CF0019D9C23
:10300000F00D1124E259FD4F1382128280911401B8
:103010009601280F311D9C9CF0019D9CF00D112400
:10302000E259FD4F4281618180810E943908839479
:10303000C7CF9C9C80019D9C100D112402591D4FEF
:10304000F8018381811509F181508383589EC00165
:103050001124648170E00E946F31FB01F595E795C2
:10306000EF77FF27E454FB4F8491E82FE7195E9E2A
:10307000C0011124B7010E946F3180910704689F3D
:10308000B0011124F8017283C1CF0E948C32B501C6
:103090000E94D3318C179D070CF0B8CFF3E06F1668
:1030A00098F00E948C32B5010E94D331F8018083E0
:1030B0000E948C32209106042695622F70E00E94B7
:1030C000D331280FF80121839C9CF0019D9CF00DC9
:1030D0001124E259FD4F128280910704893C58F077
:1030E00088EC9C9CF0019D9CF00D1124E259FD4F51
:1030F000848383838BCF8431A0F784E1F2CF0F9355
:10310000CF93DF93C4E0D4E0488159816A817B8109
:1031100088E090E00E941033288139814A815B81E8
:103120006C817D818E819F8100E20E942A32622F14
:1031300083E290E00E94FE32DF91CF910F910895DB
:10314000E4E0F4E085E0808311828FEF8283838363
:103150001482E1E0F4E082818360828384E094E081
:10316000CECF80910804833018F48F5F80930804D9
:1031700084E094E0C4CF80910804811519F0815057
:103180008093080484E094E0BACFA0E0B0E0EBECD8
:10319000F8E10C948E31D82F062F142FE22E3091A7
:1031A000040430FF35C0809105048D1308C0909150
:1031B0000604961304C090910704941729F0909187
:1031C0000304926090930304E32FE695E695AE2FF7
:1031D000B0E0A456BE4F9C91909301043C7F3430E4
:1031E000E1F46D2F702F812F0E94B207962F672F69
:1031F000482F892F0E9472088D2F80930504009319
:10320000060410930704E11419F084E094E077DFDA
:10321000CDB7DEB7E7E00C94AA31923019F41091E3
:103220000704EACF963049F3993039F3993121F701
:10323000E9518E2F8170D82EE695F0E0E45CFA4FCC
:10324000C491F12C60911601F61618F00E945808EE
:10325000D3CFFC9EC001112470E00E946F318D2FEE
:10326000D1100CC0860F209114012F0D3327331F6E
:10327000412F602F0E943908F394E4CF861BF3CFCF
:10328000E4E0F4E0818121E043816281885F7DCFC9
:10329000E4E0F4E0818121E043816281885075CFD0
:1032A000E4E0F4E0628121E1620F08F46FEF21E0D5
:1032B000438181816ACFE4E0F4E0628121E1621B15
:1032C00008F460E021E0438181815FCFE4E0F4E035
:1032D000438121E1420F08F44FEF21E062818181B7
:1032E00054CFE4E0F4E0438121E1421B08F440E0E4
:1032F00021E06281818149CFA0E1B0E0E2E8F9E11B
:103300000C948531FE01319680E1DF011D928A9592
:10331000E9F70BE110E091E5A92E92E0B92E2FEA32
:10332000422E55245394612C712C4F01730162017C
:10333000B1E14B165104610471041CF080E1C82E08
:10334000D12CA601B501C4010E94EF32AC0CBD1C0A
:103350000D2C000CEE08FF084C185D086E087F0865
:103360000150104019F76096E0E10C94A1316FEF25
:1033700085E290E00E94FE326FEF86E290E00E94CC
:10338000FE326FEF87E290E00E94FE3260E088E25A
:1033900090E00E94FE326CDDAFDF63EF85E290E0EB
:1033A0000E94FE3269E086E290E00E94FE3261E80F
:1033B00087E290E00C94FE328F929F92AF92BF9280
:1033C000CF92DF92EF92FF920F93CF93DF9388E03B
:1033D00090E00E94E5324B015C01C4E0D4E06883D8
:1033E0009982AA82BB821C821D821E821F8283E276
:1033F00090E00E94DD32282F30E040E050E060E0B5
:1034000070E080E090E000E20E940F322829392924
:103410004A295B29288339834A835B836C837D83B4
:103420008E839F83DF91CF910F91FF90EF90DF907C
:10343000CF90BF90AF909F908F9008951F921FB62E
:103440001F9211248F939F93AF93BF938091F502A6
:10345000811113C08091220290912302A091240235
:10346000B09125024196A11DB11D80932202909337
:103470002302A0932402B0932502BF91AF919F91A4
:103480008F911F901FBE1F9018952FB7F8948091B1
:10349000220290912302A0912402B09125022FBF15
:1034A000089580914603811509F0EFCF0E94020C28
:1034B000CB010895609104046695669570E04BE039
:1034C00050E087E091E00E94A332892B19F481E05B
:1034D00080930204E6DF90930603809305038091B6
:1034E000030484608093030408959091040490FF82
:1034F00031C0811581F18B3280F58F73880F880F71
:10350000909104049370892B8093040480910304A8
:10351000816080930304611519F084E094E0EFDD8D
:10352000609104046695669570E04BE050E087E09A
:1035300091E00E94A332892B91F00E94CF0881E094
:103540008093080320E04091070460910604809175
:1035500005041BCE089581E0D1CF8AE2CFCFAADF48
:10356000EECF80910404869586958F5F8B3208F0AC
:1035700081E061E0BACF80910404869586958A95B2
:1035800009F48AE261E0B1CFCF93DF93EC017DDFF4
:103590008C1B9D0BDF91CF910895A6E0B0E0E3ED89
:1035A000FAE10C9493319093490380934803811579
:1035B00020E2920730F40E94FD0F2696E2E00C9480
:1035C000AF3180EF89838A8360DF8160BC014981EC
:1035D0005A8181E090E00E942523EFCFA7E0B0E080
:1035E000E4EFFAE10C9483318C01DC0114968C91A8
:1035F000811509F4A7C061E0C801C7DA7C01809198
:10360000FA0381111DC0F8018581811509F45FC09D
:10361000E114F0E5FF0638F5E11420E2F20608F0C7
:1036200095C0E11437E0F30659F030F4C701805E2D
:103630009109089758F504C0E1145FE0F50631F5EB
:103640008091FC03811185C1E114BEE7FB0609F0FE
:10365000A3C1F8019581911509F474C091E08927FF
:103660008093FC036FC090EEE91692E5F90648F5E9
:10367000A0ECEA16A2E5FA0618F7B0E4EB16B2E5FC
:10368000FB06D0F4E114E2E5FE06D0F620910D042D
:103690008091100499E0F801A6EEB3E001900D923C
:1036A0009A95E1F7F092EE03E092ED031092F003A9
:1036B000822B8093E503C4CFC70180569245809743
:1036C000B9CF970127573C4725303105F8F6B9E7C0
:1036D000EB16BCE7FB0609F03EC02091ED033091EC
:1036E000EE03232B79F18115A1F081E00E948E0B6E
:1036F0008091E5030E94340F89E0E6EEF3E0ACE947
:10370000B3E001900D928A95E1F78091F0038093E8
:103710009B0386E0F801ACE9B3E001900D928A9535
:10372000E1F780919B038093FA038CE993E056DFE5
:103730001092FA03F8018581811104C08091E5039C
:103740000E94430F2796E2E10C949F31D801169610
:103750008C9180316FCFFAE7EF16FCE7FF0609F096
:103760006FCF811509F4CAC0A090ED03B090EE03AD
:103770002091E5032E832983BE016F5F7F4FC50132
:103780000E94D10A2C0139813F83F5EACF2EF3E064
:10379000DF2EEE24E394F12C22242A94D6011796EE
:1037A0003C90179733FE54C06D907C901197129601
:1037B0008D909C90139746145704B9F41496BC91BD
:1037C000BD83232DF60146816B2F8F810E94EB0A6A
:1037D000811559F08D810E94B304281634F4D60166
:1037E00015969C917401F92A282E48145904C9F49D
:1037F00031FE17C0F601F581FD83232DD601169603
:103800004C916F2F8F810E94EB0A811551F08D81B1
:103810000E94B30428162CF4F60194817301F92A4E
:10382000282E30FE15C0FFEF2F1212C021E0E21645
:10383000F10471F4232DD60116964C9160E08F812E
:103840000E94EB0A811521F0F60185817401F82AA6
:10385000F8E0CF0ED11C25EEC21623E0D20609F007
:103860009DCF31E0E316F104F1F59E8192959F70B2
:103870004E81942B9F7081E0403108F480E0F82E57
:10388000F294E0EFFE22F92AA11450E2B50620F5E9
:10389000A11481E0B80608F055C0EA2C8F2D8D7078
:1038A0004A2D811509F451C06AE082E998E00E942E
:1038B0009F0B282F30E02115310551F44E2D6CE07F
:1038C0008EE798E00E949F0B282F30E0811549F089
:1038D000F901FF297F0107C0C5019052811590436E
:1038E00090F1E12CF12C87E0E1EFF3E0DF011D9294
:1038F0008A95E9F7F092F903E092F8038091F803D2
:103900009091F903892B09F41DCFF8018581811568
:1039100039F08FEF0E948E0B8091F0038093EF03BC
:1039200086E0F801A1EFB3E001900D928A95E1F7EE
:103930008091EF038093FA0381EF93E04FDE1092C2
:10394000FA0300CFFB28BB24A8CF68E08AE898E000
:10395000AECF9701245031092A31310508F074CED9
:10396000D80115968C918115B9F08091FB0391E0F7
:1039700089278093FB03811109C06894F1F8C7017E
:103980000E94D10FC7010E94FD0FDCCE60E070E005
:103990008E2D0E941210D6CED80115964C9141154D
:1039A00009F4A5C4C70197578038910508F0BCC435
:1039B0001E2D103108F0C6CE6EEA71E080E090E076
:1039C00045D98111BFCEC12CD12C760111113EC039
:1039D00074E0272E8E010F5F1F4FD801E22D1D923C
:1039E000EA95E9F746015701FFEF8F1A9F0AAF0AE0
:1039F000BF0AC701B6012AD98983811509F4A2CE6D
:103A0000813009F0A2C02601370122E0420E511C8C
:103A1000611C711CC501B40119D9382E8A83811526
:103A200009F490CE8FEF830D833020F5C301B201EE
:103A30000DD98B83811511F0C80132D94601570188
:103A400033E0830E911CA11CB11C48C0BFEACB1609
:103A5000B1E0DB06E104F10409F474CEC701B6015C
:103A6000F5D8EFEFCE1ADE0AEE0AFE0A8111EECF8C
:103A70001150ACCF8BEF830D833098F54601570181
:103A800043E0840E911CA11CB11CC301B201DED81D
:103A90008B83811519F1C501B401D8D88C838115A8
:103AA000B1F0AB80BC8051E0A5165FEFB50610F019
:103AB000BA2CAA2486E0381641F097E0391611F0A6
:103AC000C50172D6C50169DD02C0C5016DD64601CA
:103AD0005701F4E08F0E911CA11CB11C750164010B
:103AE0007CCFA4E0530142013A12F8CFC301B201E6
:103AF000ADD8782E46015701B4E08B0E911CA11C65
:103B0000B11CC701B6016D5F7F4F8F4F9F4F9ED88D
:103B1000711409F417CE811509F414CE8150990B54
:103B20004FEF489F9001499F300D1124E72DE15040
:103B3000FF0B2E0F3F1F2150310980F28FE99FE0CC
:103B40000197F1F700C00000F6CFC801A9D8C6CF91
:103B500010920D049ADC88579C4E9093FF0380933B
:103B6000FE0381E08093FD03EDCDF2EBEF16F2E56D
:103B7000FF06E9F525EE30E02770332781E090E07D
:103B800001C0880F2A95EAF7209100043091FD03C7
:103B90003115E1F04115A9F0282B20930004D2CD76
:103BA000D80116968C91803110F58F2D99278F7141
:103BB00099278230910511F04297DBCF21EE30E05A
:103BC000DBCF8095822380930004BCCD322F382335
:103BD000311569F0982F90959223909300040E94DC
:103BE000B205D80115968C91811509F4ABCD809161
:103BF000FD03811509F469C0D0900D0446DC885797
:103C00009C4E9093FF038093FE03F80185818115FC
:103C100009F45BC08D2D8D79811182C0E114F0E52E
:103C2000FF0608F5E11420E4F20608F083C036EE42
:103C3000E316F10409F449C0C7019052811590427E
:103C400008F07FC0D80116968C91803108F460C0CE
:103C5000C7019927109210048D32910509F582E071
:103C60008093100472C0B0EEEB16B2E5FB0608F0CC
:103C70003FC0E0ECEE16E2E5FE0638F5F0EAEF169E
:103C8000F2E5FF06E8F420E6E21622E5F206E8F4A3
:103C9000C701925580349105C0F010921004C701FD
:103CA0008E32910508F05EC08832910508F04BC055
:103CB0008E31910508F049C004974A9780F230C0D0
:103CC00034EBE31632E5F30641F7F80195819115DF
:103CD00009F4FEC280910D048272F701E052F847A8
:103CE000EB30F10508F088C0E456FC4C0C94E6314A
:103CF00049E7E4164CE7F40630F457E7E5165CE7CD
:103D0000F50618F7CACF8BE7E8168CE7F806DCCF84
:103D10008F2D8F718431C9F2863111F41092100405
:103D20000E944D0F80910D0490910004892B809387
:103D30000D04CBCFD80116968C91803108F088CF36
:103D4000C4CFC70187CF8A9759F7809100048115A6
:103D500031F08091100492E08927809310040E9432
:103D6000D40EB3CF8C34910581F38D329240ECCFD9
:103D70008091040480FF10C08E7F8093040484E04F
:103D800094E0BDD90E94CF088091030481608093A4
:103D900003040E945808D6CC81608093040461E03B
:103DA00086958695A2DBCECC811521F0E4DBCACCCA
:103DB0008115E1F3D6DBC6CC811521F069DAC2CCDE
:103DC0008115E1F35DDABECC811521F074DABACC4D
:103DD0008115E1F365DAB6CC811521F082DAB2CC37
:103DE0008115E1F373DAAECC811521F0C4D9AACCE8
:103DF0008115E1F3B6D9A6CCF7E7EF16FCE7FF068D
:103E000009F128E7E2162CE7F20601F19701205E9E
:103E1000324520323105F8F491111DC03E2D3F711D
:103E200081E090E0AC0102C0440F551F3A95E2F7E3
:103E30007A01642F83E090E00E94FE328E2D0E9472
:103E4000E10480CC81E00E94E8044BC282E091153D
:103E500009F445C2F8CF80910C04D0900F042D2DA9
:103E600030E02095309550E028233523232B19F09E
:103E70008D2180930C045BE7E5165CE7F50649F4B9
:103E8000911509F45FCC8D2D0E94B6040E94740B2D
:103E900059CC80E4E81682E5F80608F053C0A0E2A9
:103EA000EA16A2E5FA0608F054C0E114B0E5FB06F4
:103EB00030F5E114E0E4FE0608F061C0911509F464
:103EC00077C0B1E0EB16BCE7FB0609F49DC0E3E068
:103ED000EE16ECE7FE0609F491C0E114FCE7FF06DC
:103EE00009F066C00E9428102FEF34E34CE0215007
:103EF00030404040E1F700C000000E94C10D970132
:103F0000305521153240D0F6970145E0369527957A
:103F10004A95E1F7822F8F7020910C0430E041E048
:103F200050E0082E02C0440F551F0A94E2F72423E4
:103F30003523232B19F29111A9CF10920D040E9461
:103F4000D40E00CC9701205C32452032310508F0B8
:103F5000B5CF8E2D8F7120910C0430E041E050E000
:103F6000082E02C0440F551F0A94E2F7242335237C
:103F7000232B09F4A3CF911509F4E4CB87CFD80103
:103F800016968C91803108F099CF911111C08F2D28
:103F90008F7021E030E002C0220F331F8A95E2F7D4
:103FA00040910C0450E024233523232B09F0CACB85
:103FB000D80117962D913C912115310539F1C90190
:103FC0000E94AD06F82ED80115962C9115971696DD
:103FD0003C9132953F70892F82958F70883009F41B
:103FE000A7C058F58230C8F1825F8F70823008F424
:103FF00070C060E0C8010E94C515A4CB6FEF7FEFD1
:1040000080E090E00E9418330E944010F801A080E8
:10401000B180911569F0C5010E949B15F82E682F9B
:10402000C5010E945605B5018F2D0E947115C8CF9C
:10403000C5010E947005F82EF6CF893009F4E9C059
:104040008A5F8F708230A8F6B2EFFB12F4C0892F1E
:104050008F71211509F421C1EBC0E92FEF70EE2E0D
:10406000903118F0E29480EFE8222115C9F0E114B4
:1040700069F080E28F0D883010F0F1100BC0809154
:104080000D048E2980930D040E94D40E8F2D0E9462
:10409000560FAFCF809110048E2980931004F4CF77
:1040A0008F2D0E94E60FE11409F4A3CF80E28F0D5B
:1040B000883010F0F11006C08E2D0E94B2050E94CB
:1040C000D40E97CFE094809110048E218093100439
:1040D000F6CF892F8F70907F903211F08295807F7C
:1040E000F1E0FF120EC0211531F0363008F081CF1B
:1040F0000E942B0F7ECF353008F07BCF0E943D0F02
:1041000078CF211519F0311599F3C0CF3115B1F3DE
:1041100029E3F21209C03FEF47EE53E0315040402F
:104120005040E1F700C000008F2D0E94E60F61CFE4
:10413000892F8370811136C0211129C08F2D82955E
:1041400086958770880F880F2F2D2F70082E01C03D
:10415000220F0A94EAF74F2D4071F4FE07C04FE09A
:1041600050E001C0440F8A95EAF7409596959695E0
:104170009370923091F0842F822B933031F08091A4
:104180000E04913039F0242B82230E94E1040E9416
:10419000B40B2FCF822B842BF8CF242B80910E04CD
:1041A0008227F3CF211571F190FFF1CF8F2D8295EA
:1041B00086958770880F880F2F2D2F70082E01C0CD
:1041C000220F0A94EAF74F2D4071F4FE07C04FE02A
:1041D00050E001C0440F8A95EAF740959695969570
:1041E0009370923091F0842F822B933041F0842F82
:1041F000822B8D21913019F48D2D822B842B0E94DE
:10420000E404C5CF823018F2D1CF842F822B8D25C4
:10421000F6CF9F70E92E211539F0892F0E94E8040E
:104220008F2D0E942B0FB3CF8F2D0E943D0F8E2D0F
:104230000E94F204ACCF83EFF81670F4A0EFFA16E8
:10424000C1F0B1EFFB1629F1211569F1311541F1EA
:104250008F2D0E94560F9BCFE3EFFE12F5CF80E02B
:10426000211569F29F7181E001C0880F9A95EAF7E4
:10427000C6CF211561F0353008F089CF292F2F7175
:1042800081E090E001C0880F2A95EAF7C0CF363070
:10429000F3CF892F8F71211559F20E94E80477CF4F
:1042A000892F8F71FACF311581F0F9E3FF1209C020
:1042B0002FEF37EE43E0215030404040E1F700C09F
:1042C00000008F2D0E94E60F62CF892F8F71B0CF33
:1042D00057E7E5165CE7F50609F093CD81E00E940B
:1042E000F20443E062E081E00E9489052BCA83E783
:1042F000E8168CE7F80609F425CAA2EAEA16A2E550
:10430000FA0609F45BCC08F030CCC7019052811555
:10431000904208F445CCB1EEEB16F10409F44ECC12
:10432000E5EEEE16F10425CC93E7E9169CE7F906D5
:1043300021F78091FD03811509F40ACC0E944D0FED
:1043400001CA80916104803178F480916004811504
:1043500059F0E09112042091110430915C044091D5
:104360005B0459E02E1301C008956E2F70E05E9F2C
:10437000F0011124DF01AD5EBB4F14968C911497B0
:10438000811551F111968C911197831325C08C9151
:10439000841322C015968C91159781111DC0129619
:1043A0008D919C91A0915D04B0915E048A1B9B0B42
:1043B000883C910588F4809161048F7080618093BE
:1043C0006104E75EFB4F80818F70806180838BE5A5
:1043D00094E004D90C94A805FB013196E770C2CF94
:1043E000AFE0B0E0E6EFF1E20C9487318C0186E0BB
:1043F000F801DE011A9601900D928A95E1F7F80115
:10440000F58084819BE5892E94E0992E60905F046D
:10441000611017C0811591F0F11409F412C1C8019F
:104420000E94F415811509F40CC189E0F801ABE58F
:10443000B4E001900D928A95E1F783DFFF24F394B5
:1044400055C07080A280B380D090600420915D043C
:1044500030915E04A501421B530BD11409F4C1C075
:10446000483C510508F076C0811541F380915C0409
:10447000C180E090610450E1E51608F057C0C81211
:1044800014C080915B04871110C0F11049C08E2DBB
:104490008F708061809361048BE594E09FD8809158
:1044A0006104F8018683F12C21C0F11039C040E08D
:1044B0006C2D872D0E947C0D40E06C2D872D0E9475
:1044C0007C0DF82E8111EFCF8A859B850E94E71520
:1044D000292F22952F70903470F49F70223098F01D
:1044E0009115A9F0F8019681903188F48F2D2F96BF
:1044F000EEE00C94A3312A5F2F70223060F0C801E7
:104500006DD8FD2CF3CF911511F0811579F3805EF4
:10451000883060F3F4CF803F48F3815F8330F9CF78
:1045200080916104816080936104BDCFC81238C05E
:1045300080915B04871134C0F11032C0E682C8015B
:104540004DD889E0F801ABE5B4E001900D928A9571
:10455000E1F774CFE0906104F0E1EF1648F48BE5E9
:1045600094E03CD889E0F40111928A95E9F79BCF59
:10457000811509F463CF90915C04F801818198134F
:104580000FC080915B0487110BC0F11009C0E68257
:10459000C80124D889E0F40111928A95E9F74ECF39
:1045A000C8010E94F415811509F44BC0F11409F4F7
:1045B00048C080916104803208F437CF1E821F8288
:1045C0001886198680915B0490915C049A83898394
:1045D000BC82AB826D82EF82CE0101960E94EE1A00
:1045E00024CF483C510508F0BDCF811509F426CFF2
:1045F000F11439F190915C048181981318C0809175
:104600005B04871114C08091610480FD9ACF8031D2
:1046100008F497CF8683807F803F09F490CF86810E
:10462000982F907F905F8F70892B868388CFC801E9
:104630000E94F4158111F9CE80916104816080930C
:104640006104C8010E94EE1AF9CEA1E2B0E0EBE2EB
:10465000F3E20C9491314C8F5D8F6E8F7F8F88A326
:10466000192F99A3911110921004198E1A8E1B8E76
:1046700086E0FE017C96DE01539601900D928A95AC
:10468000E1F708A1011561F00F8B188F61E0CE01F1
:1046900043960E94C51561E0CE0143960E94C51560
:1046A0000F8B188F89E0FE017396DE011A96019038
:1046B0000D928A95E1F7CE010A9692DE811128C00B
:1046C0009E85209111043091120489E0FE013A96F2
:1046D000DE01119601900D928A95E1F79115C1F0D6
:1046E000822F90E001968770992738171906D9F024
:1046F00099E0929FD0011124AD5EBB4FFE0131962F
:1047000001900D929A95E1F7809311040E94A805FB
:1047100019E08091120490911104891312C0A1969E
:10472000E4E00C94AD310E94281010921104109214
:10473000120489E0EBE5F4E0DF011D928A95E9F7C8
:10474000E7CF189FC00111248D5E9B4F49DE811574
:1047500031F38091120490E001968770992780933D
:104760001204D7CFA6E0B0E0E8EBF3E20C9491316D
:104770000E94451A8C0180914C0390914D03801743
:10478000910771F019821A820E94451ABC01498171
:104790005A8180E090E059DF10934D0300934C0361
:1047A0002696E4E00C94AD31A6E0B0E0EAEDF3E249
:1047B0000C9493319093490380934803811520E230
:1047C000920730F40E94D10F2696E2E00C94AF31AC
:1047D00080EF89838A830E94451A8160BC014981E8
:1047E0005A8181E091E031DFEFCFACE0B0E0EBEF58
:1047F000F3E20C948D3180E01CEF0DEFFF24F39475
:1048000090910E0320910D03291709F441C0E92F5F
:10481000F0E0E15FFC4F808187FBCC24C0F8D82E0C
:10482000E894D7F89F5F937090930E0390910C03D8
:104830009F5F90930C0387FD07C0DF8218870E945B
:10484000451A23E0E22E06C0DF8208870E94451A3F
:1048500032E0E32EBC0189879A87EB86FC864F8184
:1048600058858E2D91E0F1DED982C11479F00A834A
:104870000E94451ABC018B839C83ED821E82498174
:104880005A818E2D90E0E1DE81E0BACF1A83F0CF1D
:104890002C96E8E00C94A931A5E1B0E0E2E5F4E261
:1048A0000C948631FE013C968AE0DF011D928A95C8
:1048B000E9F78FE1E82E81E0F82E8F0194E2C92E0E
:1048C00091E0D92E3F01AA24A394B12C3FE1832E7D
:1048D00031E0932EF70181917F018F3F09F43EC0B3
:1048E000F894E82FE295EF70F0E021A18F70A50118
:1048F00002C0440F551F8A95E2F7CA01922F982BE8
:1049000091A392A18095892382A3789400C0E7E1C6
:10491000F1E031E0512C21912F3F79F0A22FA295A7
:10492000AF70A05EB0E08C9190E02F7002C09595C2
:1049300087952A95E2F780FF86C080E0582A330FDA
:104940008E169F0641F7F70182918F3F11F00E946A
:10495000940750EA5A95F1F7D8015C920F5F1F4F08
:10496000CE14DF0409F0B6CF4AE050E0B30188EE80
:1049700092E00E94B0329C01892B41F08AE0F30161
:10498000A8EEB2E001900D928A95E1F70091F30252
:1049900010E0025E1C4F232B09F457C081E0809386
:1049A0000D020E94451A90930C0280930B02809195
:1049B0004603FE0131967F01811509F49FC085E011
:1049C000DF011D928A95E9F780910E028A3008F086
:1049D00060C044EE53E1B701C8010E94420E811548
:1049E00009F47AC04FE054E1B701C8010E94420EB9
:1049F000811509F471C042E654E1B701C8010E9473
:104A0000420E811509F468C044EA54E1B701C801B7
:104A10000E94420E811509F45FC010920E0280912F
:104A2000F20290E045E050E0B701825E9C4F0E94A8
:104A3000B03221E020930A02892B09F041C065962B
:104A4000EFE00C94A231832F79CF80910D02811574
:104A500009F4ADCFE0900B02F0900C020E94451AD1
:104A60008E199F09059708F4A2CF45E050E068EE43
:104A700072E0C8010E94B032892B41F085E0E8EE77
:104A8000F2E0D80101900D928A95E1F710920D02A3
:104A90008ECFC0900802D09009020E94451A8C194E
:104AA0009D09843F914008F094CF80910A028115BE
:104AB00031F285E0F70111928A95E9F710920A0226
:104AC000A091F202B0E0A25EBC4F85E0F701019038
:104AD0000D928A95E1F7B3CF80910E028F3F39F4A2
:104AE0000E94451A9093090280930802DECF8F5FDF
:104AF00080930E028A3008F492CFF2CF85E0F8015D
:104B0000A9E6B4E001900D928A95E1F765E070E0C6
:104B100089E694E00E945C0B8093680488E0EBE0F7
:104B2000F3E0AFE6B4E001900D928A95E1F768E01A
:104B300070E08FE694E00E945C0B80936E0480909E
:104B4000770490907804A0907904B0907A048091D2
:104B5000040290910502A0910602B0910702881606
:104B60009906AA06BB06B1F0809204029092050253
:104B7000A0920602B09207020E94F60B861A970ACC
:104B8000A80AB90A8092420390924303A092440378
:104B9000B09245038BE0EBE7F4E0D70101900D9272
:104BA0008A95E1F7F0907C04E0907D04D0907E043B
:104BB000009184041091850410928504111509F464
:104BC0003ECF10FF0DC0898180FF1EC0909104046C
:104BD00091609093040460E0869586950E94751A12
:104BE00011FF06C020E04D2D6E2D8F2D0E94C5189F
:104BF00012FF04C0011559F00E945A1A13FF1FCF6B
:104C000081E0809308031BCF0E94D608E9CF0E9461
:104C1000CF08F4CFCDB7DEB7AA970FB6F894DEBFB2
:104C20000FBECDBF85B7806885BF85B7806885BF5B
:104C300084B7877F84BF0FB6F894A89580916000F1
:104C4000886180936000109260000FBE80E890E061
:104C50000FB6F89480936100909361000FBE81E0DD
:104C60008093740182E997E09093DB018093DA01ED
:104C70000E94F8165098589A5198599A859A869A8F
:104C8000879A0E94C50C0E94220D8091E2008460E8
:104C90008093E200789480912A03811599F08091A5
:104CA000E9001091EC008F70179511271795182BBC
:104CB0001092E9008091E80083FD0E9455101F705A
:104CC0001093E90082E084BD93E095BD9AEF97BD13
:104CD00080936E001092420310924303109244039B
:104CE000109245030E943716811102C00E94B71925
:104CF00088EC90E02091E30027FD0EC0AFE3BCE913
:104D00001197F1F700C000000197A1F70E94C50CB0
:104D100010922A0380E001C081E0809346038093D3
:104D2000470380932401811509F4E5C01092120114
:104D30008CE0809313010E945D2FEBE0F3E088E0AC
:104D4000DF011D928A95E9F78091240191E089277E
:104D5000809315038091240190931803809124017E
:104D600060E080E00E942D0B61E080E00E942D0B4E
:104D7000EFE8F1E03197F1F700C0000010E080911A
:104D80001803181708F4BDC080912401811124C0B4
:104D900085E0E5E7F1E0DE01919601900D928A95BC
:104DA000E1F785E0FE01B196AFE1B1E001900D922F
:104DB0008A95E1F788E0EBE7F1E0DE0111960190DA
:104DC0000D928A95E1F788E0FE013196A7E1B1E006
:104DD00001900D928A95E1F78091240190E0811174
:104DE00001C095E09093F30285E0891B8093F20265
:104DF0000FE111E0D8018D918D018F3F11F00E94DC
:104E00009407B1E004321B07A9F707E111E0F801AC
:104E100081918F018F3F11F00E949407F1E00F31D3
:104E20001F07A9F78AE0EEE1F3E0DF01282F1D92CA
:104E30002A95E9F7E8EEF2E0DF011D928A95E9F79D
:104E400080E090E00E94EA32833E9E4F21F40E946F
:104E5000371681112BC063EE7EEF80E090E00E9458
:104E6000183360E082E090E00E94FE3281E080939F
:104E70000E0461E083E090E00E94FE3260E074E1A5
:104E800084E090E00E9418330E94A0180E94B71995
:104E900040E050E0BA018FE090E00E94103340E023
:104EA00050E0BA0183E190E00E94103382E090E08C
:104EB0000E94DD328093F70284E090E00E94EA32A3
:104EC00090939A0380939903E7DCEFEFF6E721E0F4
:104ED000E150F0402040E1F700C00000DDDC8091AF
:104EE0001E0380FF20C06FEF7FEF80E090E00E9404
:104EF00018330E94C10D8CE080931201809313013E
:104F00001CCF60E0812F0E94410B082F61E0812FB0
:104F10000E94410BE12FF0E0EA5EFC4F880F802BEE
:104F200080831F5F2CCF83E090E00E94DD320E94DF
:104F3000E10480910F040E94C9048091F402811160
:104F400025C084E094E00E94DC1980910304836012
:104F50008093030480910404843030F40E94A018EC
:104F600084E094E00E94DC190E944A080E94CF0865
:104F70000E944F0B8091040480FF05C060E086957D
:104F800086950E94751A81E08093F4028091460311
:104F9000811103C082E30E94BC3085E291E09093CE
:104FA0006F0380936E0380912A0310E4853009F427
:104FB0007CC072DC08EF12E04EE1E42E43E0F42EF8
:104FC000D701F80191918D9122E033E02E173F0730
:104FD00009F475C09817B1F380904603D12CD7011E
:104FE000CD907D01F80191908F019C1431F19C24AA
:104FF000B12CAA24A394892D8A218115B9F081149A
:10500000A9F0B982DA820E94451A9C838B83F1E071
:10501000FD8391E08C2D8A21811101C090E09E8357
:1050200049815A816B817C818D810FDBB394AA0CFD
:1050300028E0B212E0CFF801C292D3943AE0D31242
:10504000CECF0E94020C3EC080912A03843019F119
:105050001092F50288E190E00FB6F894A89580933D
:1050600060000FBE1093600083B7817F846083BFB0
:1050700083B7816083BF7894889583B78E7F83BF21
:105080000FB6F894A89580916000886180936000C5
:10509000109260000FBE00DCEEE1F3E0819181111F
:1050A00044C593E0E832F907C9F780912A038530B7
:1050B00009F4CACF0E9428100E94B40B7ACF98132B
:1050C0008BCF50DB80914603811589F08091FD03E1
:1050D000811569F00E94451A2091FE033091FF036B
:1050E000821B930B8F3F9F4710F40E944D0F8091BE
:1050F0000204811509F46FC080910104E091040459
:10510000E695E695E81BE0930703853109F4DCC0DA
:1051100008F086C0893009F4CBC008F072C0823034
:1051200009F4B0C0863009F4B8C000ED17E031EBE7
:10513000E32E37E0F32E80910803811561F0109281
:1051400008030E94511A909306038093050310925E
:105150000A03109209030E94511A9C0180910503D1
:1051600090910603A901481B590B4F3F5F4798F5E3
:10517000409104034115B1F01092040340910203E1
:1051800050910303241B350B2F3F3F4758F4405DDC
:105190005A4850930303409302032091030428606C
:1051A00020930304C0900903D0900A03800F911F3D
:1051B000909306038093050385E093E0F70109953A
:1051C0008091090390910A03892B29F4CD2819F0C5
:1051D000F1E0F0930403F0904603F11411F005DBC5
:1051E000F82E80913303811551F010923303809192
:1051F0000D0380930E0380910B0380930C03E12C2D
:10520000A8C08F3009F091CFE695F0E0E75BF94F49
:10521000E4910E2F10E0B9E2EB2EB9E0FB2E8BCF1C
:1052200004EF11E07FE9E72E7AE0F72E843209F4EB
:1052300082CFA8F408E210E06DE1E62E6AE0F62ED7
:10524000883109F478CF833209F06FCFE4E4F6E0D7
:1052500005911591F5E9EF2EF8E0FF2E6CCF853220
:1052600009F063CF8E2F63E00E94BA31E92FF0E09E
:10527000EF5BF94FE4910E2F10E0EBEBEE2EE7E140
:10528000FE2E59CFF0E0EE5AF94FE4910E2F10E0C8
:1052900022EEE22E28E0F22E4ECFF0E0E15BF94F55
:1052A000E4910E2F10E090ECE92E98E0F92E43CF18
:1052B000E695F0E0E45BF94FE4910E2F10E087EF04
:1052C000E82E88E0F82E37CFF0E0EA5BF94FE49162
:1052D0000E2F10E0A6EAEA2EA9E0FA2E2CCF61E00C
:1052E0008E2D0E94410B182F60E08E2D0E94410BE5
:1052F000110F812B0E2D10E0D801AA5EBC4FEC914E
:105300009E2F9370891721F1EE0FEE0FE82BEC938F
:10531000809115038E0DEF70F0E0E953FE4F0D5EA6
:105320001C4FD080D8019C91D90EB8E060E0DB160C
:1053300024F4E9EFDE161CF461E00E940C0B8D2DC5
:10534000DD0C990B68E070E00E94D331D8018C939A
:10535000E39480911803E81610F2809146038115BA
:1053600011F043DAF82AF1100E94020C0E94B40BEB
:1053700090911903891721F0809319030E94F60B6D
:1053800080912A03843009F00ECE83E08093E900F7
:105390008091E80082FF07CE8091E80090E085FFD1
:1053A0000BC00E94940C50E2E52EF12C8E010F5F91
:1053B0001F4F811571F191E08091E8008B77809308
:1053C000E800911509F4EFCD00914A0310914B03C9
:1053D000E9810115110559F1EE3F09F04AC08A81B2
:1053E000833020F08550833008F043C0EA81EE30EE
:1053F00008F03FC0F0E0E955FC4CCE010196E6C74D
:105400008091F100F80181938F01F1E0EF1AF1082A
:1054100091F28091E80085FDF3CF8091E8008B77D1
:105420008093E8000E94940C811599F3C4CFE43175
:1054300048F4E11549F0E150E33130F4F0E0EB5489
:10544000FC4CC4C7EE3F91F28FEF898312C01A82E1
:1054500089E08B830EC08A81823081F08330B9F07D
:10546000813091F70E94F60BC7D76B837C838D83C5
:105470009E83CE0101960E94E40C95CD88E290E0D7
:105480000E94DD321B821C821D828E83F2CF8091AE
:10549000280390912903892B61F38AE0EEE1F3E080
:1054A000DE01139601900D928A95E1F7E2CF8A8191
:1054B000823051F66B817C818D819E819DD788E2FF
:1054C00090E00E94FE32D5CF4C816B818A810E9490
:1054D0000A159827892798279E838D83CACF2D8107
:1054E0003E813227232732274C816B818A810E949B
:1054F0007C0EBFCF0E943817BCCF8A81823869F1F9
:1055000078F48038B1F0813809F0B3CF60E08B8156
:105510000E94751A8B81811115C00E94D608A9CFEF
:10552000833809F0A6CF20E0409107046C818B817D
:1055300006C020E04B8160910604809105040E9422
:10554000C51897CF8091040481608093040460E0C3
:10555000869586950E94751A8CCF8B81809308045E
:1055600088CF8A818238E1F060F48038A1F08138F8
:1055700009F07FCF8091040480FF10C08695869546
:1055800068CF833809F075CF809105048B838091B3
:1055900006048C836ECF809107045BCF80E059CFE7
:1055A0008091080456CF0E944A0884E094E00E944B
:1055B0007F185FCF80E18A835CCF81E08A838FEAA6
:1055C00048CF0C810D3108F054CF8A809B809824FD
:1055D00089249824A12CB12C9E012F5F3F4F790183
:1055E000020F132F111D0E151F0509F442CF80E085
:1055F0003FEA831631E09306A104B10420F4C4010C
:105600008F5A9D4FDAD7D70114968C93BFEFEB1AC0
:10561000FB0AEFEF8E1A9E0AAE0ABE0AE4CF809113
:10562000280390912903892B09F423CF8C818D3194
:1056300008F01FCF882E912CA12CB12CCA80DB80C2
:10564000DC24CD24DC24E12CF12C8E010F5F1F4FD4
:10565000412C512C3201481459046A047B0408F08F
:1056600008CFFFEACF16F1E0DF06E104F10438F4D9
:10567000D80114966C91C6018F5A9D4FBFD7BFEFCA
:105680004B1A5B0A6B0A7B0AEFEFCE1ADE0AEE0AB0
:10569000FE0A0F5F1F4FDFCF0E947C19EACE83E026
:1056A0008ACF8C818D3108F0E4CE882E912CA12CEC
:1056B000B12CCA80DB80DC24CD24DC24E12CF12C4D
:1056C000412C512C32018E010B5F1F4F481459049D
:1056D0006A047B0408F0CDCE80E0F0EECF16F1E056
:1056E000DF06E104F10418F4C601899666D7D801F3
:1056F0008D938D01BFEF4B1A5B0A6B0A7B0AEFEFAC
:10570000CE1ADE0AEE0AFE0AE1CF2C81022F10E04B
:105710002D3108F0AECE8A819B8198278927982762
:105720002C01612C712C803EF1E09F0708F0A1CE86
:10573000822E912CA12CB12C40EE51E060E070E063
:105740004419550966097709421751056105710524
:1057500008F48FCE2091280330912903232B09F0E0
:105760003EC01C0129E2220E311C80FBEE24FF24E6
:10577000E0F880FF0BC0889620D79D818927982765
:10578000892781159C4711F48FEF8D83D501C401C2
:10579000840D951DA61DB71D80FF19C0680161E02D
:1057A000C61AD108CE0105968C0D9D1D9AA789A712
:1057B000C101800F911F01D7A9A5BAA59C918115A0
:1057C0009C4721F48FEFE9A5FAA580838601FE01AD
:1057D0003196EE0DFF1D2FEFE016F10638F08E0129
:1057E0000F5F1F4FC12CD12C760125C0948185817C
:1057F00081159C4711F42483258362E0E60EF11C99
:105800003296EACF80EE481681E0580661047104B2
:1058100030F4D80114966C91C2018996EFD6BFEF8F
:10582000CB1ADB0AEB0AFB0AEFEF4E1A5E0A6E0A8E
:105830007E0A0F5F1F4FC814D904EA04FB0410F35B
:1058400018CE8091280390912903892B09F411CE59
:10585000CE0101960E94E40CFFEF21EE34E0F150FE
:1058600020403040E1F700C0000043CB88E0E4E88E
:10587000F1E0DE01919601900D928A95E1F7FE012B
:1058800032968FE1DF011D928A95E9F786E08983E0
:1058900088E07F96DE01159605CE88E2898382E056
:1058A0008A831B821C82E5CD0B811C81012E000C9A
:1058B000220B330B45E0000F111F221F331F4A95A7
:1058C000D1F7B901A801405E5F4F6F4F7F4F40177E
:1058D00051076207730708F4CCCD0832B2E01B070A
:1058E0002105310508F0C5CD4932E2E05E076105CA
:1058F000710520F048E252E060E070E0401B510B7F
:10590000B8016A5A794F16D6B4CD1B810C8140E09C
:10591000602F812F0E9438159827892798279A830E
:10592000898341E0602F812F0E94381598278927AD
:1059300098279C838B839DCD2E813F812C37310509
:1059400069F032272327322741E08D81811101C080
:1059500040E06C818B810E94A20E8BCD8091280348
:105960009091290320E03CE7892B71F720E030E09B
:10597000EBCF4AE150E06FEF70E0CE01079606D61C
:105980008091280389830A8381E08B831C8287E0CE
:105990008D8386E07ACD81E090E090934B038093F5
:1059A0004A0382E390E090931D0380931C030E94BE
:1059B000451A90931B0380931A035BCD01151105C3
:1059C00081F1D0901F03C0902503E0901A03F0905E
:1059D0001B030E94451A8E199F098536910540F1D7
:1059E000C6FE26C0D0FE24C00E94451A90931B0319
:1059F00080931A0380911C0390911D03019790934B
:105A00001D0380931C03892B61F410924B031092A9
:105A10004A0381E090E0909329038093280300E0FB
:105A200010E08091280389830A8380911C0311CDA3
:105A300082E390E090931D0380931C03F2CF1092B9
:105A400029031092280315CD40E250E06FEF70E07B
:105A50009DD50FCD2B81273071F0283049F12111D0
:105A600008CD2FE1DC011D922A95E9F788E08C83AF
:105A700083E088A3FECC2C8166E0CE018196FC01F8
:105A8000362F11923A95E9F7283080F4629FB001E1
:105A900011246F5D7D4F46E050E07FD580E0898323
:105AA00086E0FE01B196DE011296FCCC8FEFF7CFB7
:105AB0006C8186E0FE013596DE01919601900D9293
:105AC0008A95E1F789A19AA18115ACE79A0741F47B
:105AD0002091280330912903232B11F480E090E0DA
:105AE0009AA389A38BA19CA18115BCE79B0741F4D4
:105AF0002091280330912903232B11F480E090E0BA
:105B00009CA38BA38FEF683060F4E6E06E9FB0013A
:105B100011246F5D7D4F46E050E0CE0181968CD51B
:105B200080E089830E94F816A4CC8091F60281154A
:105B300009F4BBCAA0E1A9BDB2E1B9BD09B400FE38
:105B4000FDCF8091D8008F7D8093D8008091E000B8
:105B500082608093E0008091E00081FDFCCF0E9494
:105B60002810A3CA78941F921FB61F9211248F93F6
:105B70009F93AF93BF938091220290912302A091B3
:105B80002402B09125020196A11DB11D809322022D
:105B900090932302A0932402B0932502BF91AF916A
:105BA0009F918F911F901FBE1F9018951F920F926B
:105BB0000FB60F9211242F933F934F935F936F93E0
:105BC0007F938F939F93AF93BF93EF93FF938091B6
:105BD000E10082FF09C08091E20082FF05C0809150
:105BE000E1008B7F8093E1008091DA0080FF24C088
:105BF0008091D80080FF20C08091DA008E7F809352
:105C0000DA008091D90080FFA9C080E189BD82E1DE
:105C100089BD09B400FEFDCF81E080932A03809105
:105C20001102811109C00E94C50C0E94220D8091B1
:105C3000E20084608093E2008091E10080FF1AC05E
:105C40008091E20080FF16C08091E2008E7F8093F9
:105C5000E2008091E20080618093E2008091D800B0
:105C600080628093D80019BC85E080932A0383E08A
:105C7000809374018091E10084FF2FC08091E20045
:105C800084FF2BC080E189BD82E189BD09B400FE9B
:105C9000FDCF8091D8008F7D8093D8008091E10066
:105CA0008F7E8093E1008091E2008F7E8093E200FE
:105CB0008091E20081608093E20080911002811562
:105CC00009F452C084E080932A0380912A0384302F
:105CD00009F052C082E0809374018091E10083FF5B
:105CE0002CC08091E20083FF28C08091E100877F73
:105CF0008093E10082E080932A0310921002809149
:105D0000E1008E7F8093E1008091E2008E7F80939E
:105D1000E2008091E20080618093E20042E060E076
:105D200080E00E94F20C8091F00088608093F00087
:105D300081E08093740180937301FF91EF91BF9193
:105D4000AF919F918F917F916F915F914F913F9113
:105D50002F910F900FBE0F901F90189519BC1092A5
:105D60002A031092110268CF8091E30087FF02C0DE
:105D700083E0A9CF81E0A7CF81E0ADCF1F920F9242
:105D80000FB60F921124EF92FF920F931F932F9350
:105D90003F934F935F936F937F938F939F93AF93B3
:105DA000BF93CF93EF93FF9309EE10E0F80180814A
:105DB000C091EC008F70C795CC27C795C82B108277
:105DC00080EFE82EF12CF7018081877F8083789423
:105DD0000E945510F8011082F7018081886080834D
:105DE000CF70F801C083FF91EF91CF91BF91AF9138
:105DF0009F918F917F916F915F914F913F912F91E3
:105E00001F910F91FF90EF900F900FBE0F901F907A
:105E10001895FF920F931F93CF93DF93182FEB01E9
:105E20001092BC0084EA8093BC000E94451A082F9F
:105E3000F92E8091BC0087FF28C08091B900887F2F
:105E4000883029F08091B900887F803199F51093CE
:105E5000BB0084E88093BC000E94451A182F092FCC
:105E60008091BC0087FF1EC02091B900287F80E090
:105E700090E0283199F081E090E0203411F480E046
:105E800090E091958195910909C0802F9F2D0E94E6
:105E9000C41AC817D90768F68EEF9FEFCDB7DEB7E3
:105EA000E5E05AC2812F902F0E94C41AC817D90763
:105EB000B8F6F2CF8FEF9FEFF1CF1092B90088E4E0
:105EC0008093B80008950F931F93CF93DF93EB0156
:105ED0008093BB0084E88093BC000E94451A182F71
:105EE000092F8091BC0087FF11C02091B900287F45
:105EF00081E090E0283211F480E090E09195819566
:105F00009109DF91CF911F910F910895CF3FDC0749
:105F100041F3812F902F0E94C41AC817D90708F7A0
:105F20008EEF9FEFEECF0F931F93CF93DF93EC0194
:105F300084EC8093BC000E94451A182F092F809191
:105F4000BC0087FF08C08091BB0090E0DF91CF913B
:105F50001F910F910895CF3FDC0789F3812F902F78
:105F60000E94C41AC817D90750F78EEF9FEFEECFE3
:105F70000F931F93CF93DF93EC0184E88093BC00D1
:105F80000E94451A182F092F8091BC0087FF08C076
:105F90008091BB0090E0DF91CF911F910F91089508
:105FA000CF3FDC0789F3812F902F0E94C41AC817B6
:105FB000D90750F78EEF9FEFEECFA0E0B0E0E2EE12
:105FC000FFE2A5C1682E962E5A01690178010E9450
:105FD000451A782E892E0431110518F10F3F10074C
:105FE00019F1C80164E170E07AD1162F072F612FF3
:105FF000702F862D0EDFEC01892BC1F0FFEFEF161D
:10600000FF06A9F3872D982D0E94C41AE816F906F9
:1060100070F784E98093BC00CE01CDB7DEB7EEE027
:1060200092C111E000E0E3CF15E0FCCFB701892D6C
:106030004ADFEC018501CA0CDB1C0C151D0549F378
:10604000209739F7B701F80181918F013CDFEC010E
:10605000F4CFA0E0B0E0EEE2F0E359C1982E862E36
:106060006A01590178010E94451A3C010431110569
:1060700038F10F3F100739F1C80164E170E02FD10A
:10608000162F072F612F702F892DC3DEEC01892B6E
:10609000E1F0FFEFEF16FF06A9F3C3010E94C41A57
:1060A000E816F90678F784E98093BC00CE011C1647
:1060B0001D0614F480E090E0CDB7DEB7EEE043C1FA
:1060C00011E000E0DFCF15E0FCCFB701882DFBDE4B
:1060D000EC01892B41F7689490F80E94451A782EBC
:1060E000892E84E1E816F10438F1EFEFEE16FE0692
:1060F00031F1C70164E170E0F2D0162F072F612F54
:10610000702F892D86DEEC01892BD9F400E010E098
:10611000F1E0AF1AB1080A151B05F8F4D7FDC3CF9B
:10612000C70101DFEC0197FD04C0F601E00FF11F8C
:1061300080830F5F1F4FEFCF11E000E0E0CF15E04D
:10614000FCCF8FEFE816F806D1F2872D982D0E942C
:10615000C41AE816F90698F6D9CFD7FDA4CFC7011F
:1061600007DFEC0197FD05C0CA0CDB1CF60180833C
:106170009ACFCEEFDFEF97CF8093BA0085EC809374
:10618000BC0008951F920F920FB60F9211242F9307
:106190003F934F935F936F937F938F939F93AF93AF
:1061A000BF93CF93DF93EF93FF938091B900982F24
:1061B000987F9038F1F038F4911509F48DC090363D
:1061C00099F081E034C0887E883AD9F7E09165047F
:1061D000F0E0E959FB4F80818093BB00809165041A
:1061E0008F5F80936504EDCF109264041092660473
:1061F000E8CF80916404811139C08091BB00809305
:106200006504809165048F3178F11092650480E017
:1062100091E09093640440916504209132013091A3
:1062200033014217130609F090E0909366049091B1
:10623000BC008295880F880F807C892B85688093AD
:10624000BC00FF91EF91DF91CF91BF91AF919F91F2
:106250008F917F916F915F914F913F912F910F900F
:106260000FBE0F901F90189581E0D2CFE09165048A
:10627000F0E08091BB00E959FB4F80838091650479
:106280008F5F8093650480916604811509F499CF2E
:10629000C091D701D091D801A88188E0A802D0018F
:1062A0001124AF5CBE4F1696ED91FC911797309775
:1062B00009F487CF14962D913C9115972C0F3D1F13
:1062C00011966D917C9112976C0F7D1F13964C91D6
:1062D00013978C91099575CF1092BC0072CFAA1BB1
:1062E000BB1B51E107C0AA1FBB1FA617B70710F0C1
:1062F000A61BB70B881F991F5A95A9F780959095F3
:10630000BC01CD0108952F923F924F925F926F9200
:106310007F928F929F92AF92BF92CF92DF92EF9235
:10632000FF920F931F93CF93DF93CDB7DEB7CA1BB6
:10633000DB0B0FB6F894DEBF0FBECDBF09942A88E1
:10634000398848885F846E847D848C849B84AA8489
:10635000B984C884DF80EE80FD800C811B81AA8116
:10636000B981CE0FD11D0FB6F894DEBF0FBECDBFE1
:10637000ED010895992778E0880F991F961708F086
:10638000961B881F7A95C9F78095089587FB082E7C
:10639000062687FD819567FD6195ECDF0EF49195EA
:1063A00007FC8195089597FB072E16F4009406D0FC
:1063B00077FD08D094DF07FC05D03EF490958195D9
:1063C0009F4F0895709561957F4F0895EE0FFF1FC1
:1063D0000590F491E02D0994082E8170069406949E
:1063E000811D0694811D0694811D0694811D0694CD
:1063F000811D0694801D08956927962769277827AF
:106400008727782708957DD1332312F48A1B9B0BAD
:1064100001C077D1B7FF0895821B930B0895002E1A
:10642000083090F0982F872F762F652F542F432F09
:10643000322F22270850F4CF220F331F441F551F3D
:10644000661F771F881F991F0A95B2F7002D0895C0
:1064500097FD1094002E083098F00850232F342F09
:10646000452F562F672F782F892F912DF4CF159414
:10647000979587957795679557954795379527957C
:106480000A95AAF71124002D08958F929F92AF923A
:10649000BF92CF92DF92EF92FF92CF93DF93EC0106
:1064A000688179818A819B816115710581059105DA
:1064B00021F464E279ED8BE597E02DE133EF41E0E3
:1064C00050E0D1D049015A019B01AC01A7EAB1E4E7
:1064D000E6D06B017C01ACEEB4EFA5019401EBD0EA
:1064E000DC01CB018C0D9D1DAE1DBF1DB7FF03C090
:1064F0000197A109B04888839983AA83BB839F77BA
:10650000DF91CF91FF90EF90DF90CF90BF90AF9051
:106510009F908F900895B9CF80E091E0B6CFA0E032
:10652000B0E08093000190930101A0930201B09329
:1065300003010895FB01DC0102C005900D9241505A
:106540005040D8F70895FC014150504030F0019080
:106550000616D1F73197CF01089588279927089516
:10656000FB01DC0104C08D910190801921F44150A0
:106570005040C8F7881B990B0895FB01DC0102C04D
:1065800001900D9241505040D8F70895DC0101C0B0
:106590006D9341505040E0F70895DC01CB01FC01C0
:1065A000F999FECF06C0F2BDE1BDF89A319600B46C
:1065B0000D9241505040B8F70895F999FECF92BD21
:1065C00081BDF89A992780B50895A6E1B0E044E02E
:1065D00050E0E5CFA8E1B0E042E050E0E0CFDC01E0
:1065E000A40FB51F4150504040F0CB01840F951FC0
:1065F0002E9105D041505040D8F70895262FF99993
:10660000FECF92BD81BDF89A019700B4021639F011
:106610001FBA20BD0FB6F894FA9AF99A0FBE0895E2
:106620000396272FECDFEADF252FE9DF242FE7CFC2
:106630000196272FE4DFE2CFDC01CB0102C02D91D0
:1066400005D041505040D8F70895262FF999FECF34
:106650001FBA92BD81BD20BD0FB6F894FA9AF99A7F
:106660000FBE01960895052E97FB16F400940FD0E7
:1066700057FD05D024D007FC02D046F408C0509541
:106680004095309521953F4F4F4F5F4F089590951E
:106690008095709561957F4F8F4F9F4F089531D0B2
:1066A000A59F900DB49F900DA49F800D911D112466
:1066B0000895B7FFF4CFF3DF821B930B0895A1E297
:1066C0001A2EAA1BBB1BFD010DC0AA1FBB1FEE1F6C
:1066D000FF1FA217B307E407F50720F0A21BB30BB7
:1066E000E40BF50B661F771F881F991F1A9469F733
:1066F00060957095809590959B01AC01BD01CF018F
:106700000895A29FB001B39FC001A39F700D811D8A
:106710001124911DB29F700D811D1124911D0895AA
:10672000F894FFCF321158115E1158115E11B0115B
:10673000D1115E11D712E412B81ED41ED81EDC1E71
:10674000E01EE41EE81EEC1EF01EF41EF81E362CA1
:106750004D2C542C852C9C2CB92CCB2CDE2C1F2D95
:10676000242D392A392A392A2A2D272A2B2A572A31
:10677000642A6F2A7A2A7D2AB12AD32A242A212C34
:10678000DA2ADD2AE12A0F2B4C2B4F2B512B852B9C
:106790000100000001010201191A1B1C1D1E1F200F
:1067A0002122001800181836666794929395FFF01E
:1067B0003534979601F30B270E3D0E1A0C1B0C1E59
:1067C0000E010000000000000000000001010000B8
:1067D00000000000050200000000000001070000AA
:1067E000000000000808000000000000000000ADEC
:1067F0000704100000000000000B1400000000005F
:106800000000000100F035349796003666679492D8
:1068100093953700E52B480A60E25D310044223B46
:106820000901E700AC000F02280248020001020241
:1068300002020606060909090909090F0F0F0F0FC1
:106840000F151515181919191919191919191923C5
:106850002425252525252500FF0100010000FFFF37
:0A6860000000010001FF00670400C2
:00000001FF
